:020000040000FA
:0600000023EF36F01200B0
:0600080004EF08F01200F5
:060018000CEF08F01200DD
:0610000023EF36F01200A0
:061008001CEF08F01200CD
:061018006CEF08F012006D
:06102A000100726C0000E1
:08103000E901000015000000B9
:08103800DACFE4FFE2CFDAFF9A
:10104000E9CFE4FFEACFE4FFF6CFE4FFF7CFE4FF18
:10105000F5CFE4FFF3CFE4FFF4CFE4FFFACFE4FFF2
:1010600000EE20F0140EE80403E3EECFE4FFFBD71C
:1010700000EE00F0200EE80403E3EECFE4FFFBD720
:10108000E6525EEC25F0F2A403D0F294CEEC16F01A
:10109000E55200EE1FF0200EE80403E3E5CFEDFF7C
:1010A000FBD700EE33F0140EE80403E3E5CFEDFFC9
:1010B000FBD7E5CFFAFFE5CFF4FFE5CFF3FFE5CFB0
:1010C000F5FFE5CFF7FFE5CFF6FFE5CFEAFFE5CF88
:1010D000E9FFE5CFDAFF1100D8CFE4FFE0CFE4FF6E
:1010E000E46EDACFE4FFE2CFDAFFE9CFE4FFEACF44
:1010F000E4FFF6CFE4FFF7CFE4FFF5CFE4FFF3CF53
:10110000E4FFF4CFE4FFFACFE4FF00EE20F0140E8A
:10111000E80403E3EECFE4FFFBD700EE00F0200E7F
:10112000E80403E3EECFE4FFFBD7E6529EA003D032
:101130009E9037EC22F0E55200EE1FF0200EE804FE
:1011400003E3E5CFEDFFFBD700EE33F0140EE80428
:1011500003E3E5CFEDFFFBD7E5CFFAFFE5CFF4FFE3
:10116000E5CFF3FFE5CFF5FFE5CFF7FFE5CFF6FFDE
:10117000E5CFEAFFE5CFE9FFE5CFDAFFE550E5CFC0
:10118000E0FFE5CFD8FF1000D9CFE6FFE1CFD9FFD0
:10119000060EE126E5DBCCEC2DF00001AD5101E1BE
:1011A00081D2AD6B7BEC1AF0050EC26E96EC15F099
:1011B0002EC227F02FC228F030C229F031C22AF007
:1011C0007EEC2FF028C0AFF129C0B0F12EC299F10A
:1011D0002FC29AF130C29BF131C29CF195C12CF023
:1011E00096C12DF097C12EF098C12FF02EC227F096
:1011F0002FC228F030C229F031C22AF0F3EC2EF0D1
:1012000027C099F128C09AF129C09BF12AC09CF10E
:101210002C6A2D6A7A0E2E6E440E2F6EA0EC2EF0E4
:1012200027C000F028C001F029C002F02AC003F056
:10123000BBC029F0E3EC2DF027C004F028C005F076
:1012400029C006F02AC007F027C02CF028C02DF0D6
:1012500029C02EF02AC02FF000C027F001C028F0CE
:1012600002C029F003C02AF0F3EC2EF0020E27C0D2
:10127000DBFF030E28C0DBFF040E29C0DBFF050ED9
:101280002AC0DBFF02012D5101E0ABD02C51010A35
:1012900056E0010A4EE0FF0A01E0A3D00CC22CF098
:1012A0000DC22DF00EC22EF00FC22FF099C127F003
:1012B0009AC128F09BC129F09CC12AF009EC2EF0BC
:1012C00027C000F028C001F029C002F02AC003F0B6
:1012D00008C22CF009C22DF00AC22EF00BC22FF06A
:1012E000A0EC2EF027C099F128C09AF129C09BF1FB
:1012F0002AC09CF1020EDBCF00F0030EDBCF01F021
:10130000040EDBCF02F0050EDBCF03F000C02CF0A3
:1013100001C02DF002C02EF003C02FF09DC127F0B8
:101320009EC128F09FC129F0A0C12AF00AEC2EF03E
:1013300050D00101996B9A6B9B6B9C6B52D004C28D
:101340002CF005C22DF006C22EF007C22FF099C175
:1013500027F09AC128F09BC129F09CC12AF009EC22
:101360002EF027C000F028C001F029C002F02AC0EA
:1013700003F000C22CF001C22DF002C22EF003C215
:101380002FF0A0EC2EF027C099F128C09AF129C0C7
:101390009BF12AC09CF1020EDBCF00F0030EDBCFE5
:1013A00001F0040EDBCF02F0050EDBCF03F000C02E
:1013B0002CF001C02DF002C02EF003C02FF09DC113
:1013C00027F09EC128F09FC129F0A0C12AF009ECA6
:1013D0002EF027C09DF128C09EF129C09FF12AC0A0
:1013E000A0F12C6A2D6A2E6A2F6A99C127F09AC142
:1013F00028F09BC129F09CC12AF0ADEC2FF0010A26
:1014000016E12C6A2D6A2E6A3F0E2F6E99C127F0C5
:101410009AC128F09BC129F09CC12AF00AEC2EF059
:101420007EEC2FF028C0DEFF29C0DDFF02D0DE6A8F
:10143000DD6A0001B151080DF3CFE9FFF4CFEAFFF7
:10144000710EE926000EEA22030EE926000EEA22BA
:10145000EF50800B800803E1800EB011B06FB151E6
:10146000080DF3CFE9FFF4CFEAFF710EE926000E75
:10147000EA22030EE926000EEA22010EDBCFEFFF7F
:10148000B151080DF3CFE9FFF4CFEAFF710EE92661
:10149000000EEA22020EE926000EEA22DFCFEFFF5D
:1014A000B151080DF3CFE9FFF4CFEAFF710EE92641
:1014B000000EEA22030EE926000EEA22EF50800910
:1014C000E66EB151080DF3CFE9FFF4CFEAFF710EDC
:1014D000E926000EEA22030EE926000EEA22E55272
:1014E000E750EF6EFF0E02012C5D23E10001B151C8
:1014F000080DF3CFE9FFF4CFEAFF710EE926000EE5
:10150000EA22030EE926000EEA22EF504009E66EB9
:10151000B151080DF3CFE9FFF4CFEAFF710EE926D0
:10152000000EEA22030EE926000EEA22E552E750F9
:10153000EF6E2C6A2D6A2E6A3F0E2F6E9DC127F02A
:101540009EC128F09FC129F0A0C12AF00AEC2EF01C
:101550007EEC2FF028C0DEFF29C0DDFF0001B15175
:10156000080DF3CFE9FFF4CFEAFF710EE926000E74
:10157000EA22010EE926000EEA22010EDBCFEFFF80
:10158000B151080DF3CFE9FFF4CFEAFF710EE92660
:10159000000EEA22DFCFEFFFB151080DF3CFE9FFD4
:1015A000F4CFEAFF710EE926000EEA22040EE926C6
:1015B000000EEA2260C0EFFFB151080DF3CFE9FF42
:1015C000F4CFEAFF710EE926000EEA22050EE926A5
:1015D000000EEA2261C0EFFFB151080DF3CFE9FF21
:1015E000F4CFEAFF710EE926000EEA22060EE92684
:1015F000000EEA2262C0EFFFB151080DF3CFE9FF00
:10160000F4CFEAFF710EE926000EEA22070EE92662
:10161000000EEA2263C0EFFF060EB15D02E2B12BBD
:1016200041D0B16B090EC26E3BEC1BF02C6A2D6AE7
:10163000FA0E2E6EC30E2F6E2EC227F02FC228F088
:1016400030C229F031C22AF0ADEC2FF0010A19E1C5
:101650002C6A2D6AFA0E2E6E430E2F6E2EC227F0C4
:101660002FC228F030C229F031C22AF00AEC2EF045
:1016700027C08DF128C08EF129C08FF12AC090F1CA
:1016800005D001018D6B8E6B8F6B906B250EC26E3A
:101690003BEC1BF02EC2F8F12FC2F9F130C2FAF187
:1016A00031C2FBF10001AB5101E14CD10101F72B3B
:1016B0001E0EF75D02E1ECEC1CF001018C2B010128
:1016C000F55109E08450080B04E01E0E01018C5D09
:1016D00002E12FEC17F02C6A800E2D6EBB0E2E6EE1
:1016E000430E2F6EF8C127F0F9C128F0FAC129F096
:1016F000FBC12AF0ADEC2FF0010A01E18B80010162
:10170000ED5113E12C6A2D6AAF0E2E6E430E2F6E33
:10171000F8C127F0F9C128F0FAC129F0FBC12AF07D
:10172000B6EC2FF0010A01E18B900001AF5101E10D
:10173000E6D0D30E2C6E570E2D6E350E2E6E3B0E50
:101740002F6E99C127F09AC128F09BC129F09CC146
:101750002AF0F3EC2EF027C000F028C001F029C0D9
:1017600002F02AC003F027C02CF028C02DF029C0B9
:101770002EF02AC02FF0A1C127F0A2C128F0A3C1EA
:1017800029F0A4C12AF00AEC2EF027C0A1F128C04C
:10179000A2F129C0A3F12AC0A4F17EEC2FF028C049
:1017A000FCF129C0FDF12C6AFC0E2D6E7F0E2E6E11
:1017B000460E2F6EA1C127F0A2C128F0A3C129F0C7
:1017C000A4C12AF0ADEC2FF0010A26E12C6A2D6AA3
:1017D000200E2E6E410E2F6EA1C127F0A2C128F05F
:1017E000A3C129F0A4C12AF0A0EC2EF027C000F07C
:1017F00028C001F029C002F02AC003F02C6A2D6A2B
:10180000800E2E6E460E2F6E0AEC2EF07EEC2FF020
:1018100028C0FCF129C0FDF1800E2C6EFD0E2D6E4E
:101820001F0E2E6E480E2F6EA1C127F0A2C128F008
:10183000A3C129F0A4C12AF0ADEC2FF0010A25E1E3
:101840002C6A2D6AC80E2E6E420E2F6EA1C127F093
:10185000A2C128F0A3C129F0A4C12AF0A0EC2EF067
:1018600027C000F028C001F029C002F02AC003F010
:101870002C6A2D6A2E6A470E2F6E0AEC2EF07EEC33
:101880002FF028C0FCF129C0FDF1E00E2C6EFC0EFB
:101890002D6EC70E2E6E490E2F6EA1C127F0A2C16C
:1018A00028F0A3C129F0A4C12AF0ADEC2FF0010A61
:1018B00026E12C6A2D6A7A0E2E6E440E2F6EA1C17F
:1018C00027F0A2C128F0A3C129F0A4C12AF0A0ECFE
:1018D0002EF027C000F028C001F029C002F02AC075
:1018E00003F02C6A2D6A400E2E6E470E2F6E0AEC06
:1018F0002EF07EEC2FF028C0FCF129C0FDF1010193
:10190000F55112E1F22B0F0EF25D0EE1F26BF32BAB
:10191000000EF4230B0EF31905E1F45103E1010E5F
:10192000F36FF46BC9EC1FF00001BC2B000EBD235C
:10193000BE2BBF23C02BC123C22BC323D6EC21F067
:101940000001AB6B030ED76F0101F55107E10001F8
:10195000C72B04E16AEC21F0C0EC21F0E0D91DD4E2
:10196000D9CFE6FFE1CFD9FF060EE1260001110E27
:10197000706FC9EC1FF00001C451006E016AFF0EC8
:10198000001805E1015003E10101010EF56FF00EB1
:101990000001BC6FBD6BE60EBE6FBF6BD20EC06F99
:1019A000C16BC80EC26FC36BBFCF65F0D6CF64F0FA
:1019B000CFCF67F0CECF66F0CCCF69F0CBCF68F059
:1019C000B3CF6BF0B2CF6AF0BCCF6DF0BBCF6CF091
:1019D000010EC26E150EC16E950EC06E0F0E926E88
:1019E000946AD59AD596F184F28ACD8ACD889F9053
:1019F000CD8EF28CF28ED08EA69C606B616B626B8A
:101A0000636BB16BB269B06B190EAC6F040EAE6F45
:101A10006451140A01E1ABD0060A01E18DD01B0A22
:101A200070E0020A51E00E0A34E0060A1EE0010AE4
:101A300001E0B9D00101D00E066F070E076F200E2E
:101A4000086F4E0E096F9C0E916F400E926F9C0EA8
:101A5000936F3E0E946FC00EAD6F5D0EAE6FD30EE2
:101A6000956F590E966F0C0E9BD00101B80E066F44
:101A70000B0E076F400E086F9C0E096F916F400EA2
:101A8000926F1C0E936F3F0E946FC80EAD6FAF0E2A
:101A900067D00101880E066F130E076F200E086FC6
:101AA0004E0E096F9C0E916F400E926F9C0E936FBD
:101AB0003E0E946FC00EAD6F5D0EAE6FD20E956F81
:101AC0006F0E966FAF0E6CD00101100E066F270ED1
:101AD000076F500E086F460E096F890E916FA00EAA
:101AE000926F8C0E936F3E0E946FAC0EAD6F580ECE
:101AF000AE6FD20E956F6F0E966F2F0E976F400ED2
:101B000051D00101D00E066F070E076F100E086F3F
:101B1000270E096F9B0E916F400E926F1C0E936FF4
:101B20003E0E946F500EAD6F460EAE6F820E956FE7
:101B3000390E966F060E34D00101B80E066F0B0EEB
:101B4000076F080E086FCF0E096FCE0E916F080E4B
:101B5000926F4F0E936F3F0E946F900EAD6FE20E2B
:101B6000AE6F150E956F930E966F480E19D001014A
:101B7000C40E066F090E076F600E086FEA0E096F3C
:101B8000916F600E926F6A0E936F3F0E946FE80E26
:101B9000AD6FFD0EAE6F8A0E956FCD0E966F270E50
:101BA000976F3F0E986FA69E0F0EA96EA680A85045
:101BB00001010A6F0B6BA4EC1DF0080EA96EA68044
:101BC000A8CFBBF0010EA96EA680A8500001645DED
:101BD000FCE1030EA96EA680A850665DFDE1050E2E
:101BE000A96EA680A850685DFDE1070EA96EA680CB
:101BF000A8506C5DFDE16751DE6EDD6A6651026ED4
:101C0000036A286A010E296EDECF2DF0DDCF2EF09B
:101C100060EC2FF026500224006E27500320016E46
:101C200000C0DEFFDD6E00016951E66ED950020F83
:101C3000E96EDACFEAFFE552E750EE6EED6A6851E1
:101C4000026E036A286A010E296E020EDBCF2DF0A8
:101C5000030EDBCF2EF060EC2FF026500224006E36
:101C600027500320016E020E00C0DBFF030E01C0EF
:101C7000DBFF00016D51E66ED950040FE96EDACF3B
:101C8000EAFFE552E750EE6EED6A6C51026E036AB0
:101C9000286A010E296E040EDBCF2DF0050EDBCF76
:101CA0002EF060EC2FF026500224006E2750032007
:101CB000016E040E00C0DBFF050E01C0DBFF020E4B
:101CC000DBCF02F0030EDBCF03F0DE500224006E08
:101CD000DD500320016EDB0E001AA50E011A040E62
:101CE000DB500018ECE1050EDB500118E8E111D8DB
:101CF000D2EC24F00101F55102E02FEC17F0060EB2
:101D0000E15C02E2E16AE552E16EE552E7CFD9FF1C
:101D100012000101E96BEA6BEB6BEC6B1200D9CF9F
:101D2000E6FFE1CFD9FF080EE126200E0201E76EA3
:101D30003E19E8AE02D0E73402D0E7503E5D03E33F
:101D40006D50020B02E08CEF15F00101E951EA1130
:101D500002E1000E08D0E9C1E9FFEAC1EAFFEF5055
:101D6000800B01E0010E000902E08CEF15F0050187
:101D700000511A0A02E167EF15F0030A02E155EF7C
:101D800015F0010A02E17AEF13F00F0A02E12CEFDD
:101D900013F0010A01E1C3D3030A01E191D3010A5F
:101DA00001E182D3070A01E170D3010A01E14DD3B9
:101DB000030A01E144D3010A01E13BD31F0A01E117
:101DC00032D3030A01E18BD2070A01E1C5D1010A2E
:101DD00001E1B7D1020A01E1ADD10F0A01E1A5D1BC
:101DE000010A01E19AD1030A01E1DBD0010A1AE0FC
:101DF000070A12E0010A02E079EF15F0EBEC16F0A9
:101E000021EC17F00001010EAF6F0001400EB06F22
:101E100055EC1DF079EF15F02FEC17F055EC1DF097
:101E200079EF15F00001B56BB1C0B4F0070E0001F9
:101E3000B45D15E255EC1AF00001B451080DF3CF72
:101E4000E9FFF4CFEAFF710EE926000EEA22030E45
:101E5000E926000EEA22EF6A0001B42BE7D7000161
:101E6000B46B0001B1510001B45D15E055EC1AF0FE
:101E70000001B451080DF3CFE9FFF4CFEAFF710E72
:101E8000E926000EEA22030EE926000EEA22EF6A96
:101E90000001B42BE6D70001B151020A12E0030A97
:101EA00001E026D0A5C127F0A6C128F0A7C129F0DE
:101EB000A8C12AF07EEC2FF028C0DEFF29C0DDFF8C
:101EC00023D0800E2C6E2D6A2E6A470E2F6EF8C11D
:101ED00027F0F9C128F0FAC129F0FBC12AF00AEC79
:101EE0002EF07EEC2FF028C0DEFF29C0DDFF0CD0E5
:101EF000000E0101AF25006E400E0101B021016E00
:101F000000C0DEFF01C0DDFF010EDBCF78F5DFCFC3
:101F100079F50001B1A116D02C6A2D6A2E6A3F0E08
:101F20002F6EB7C027F0B8C028F0B9C029F0BAC0EA
:101F30002AF00AEC2EF07EEC2FF028C0DEFF29C03C
:101F4000DDFF17D02C6A010E2D6E800E2E6E460E10
:101F50002F6E8DC127F08EC128F08FC129F090C15E
:101F60002AF00AEC2EF07EEC2FF028C0DEFF29C00C
:101F7000DDFF010EDBCF7AF5DFCF7BF5FDC17CF510
:101F8000FCC17DF5B2C07EF5B0C07FF57F0E0001CB
:101F9000B0150001B06F55EC1DF001018C6B79EFAD
:101FA00015F0F3C140F5C4C041F52C6A2D6A2E6AC4
:101FB0003F0E2F6E9DC127F09EC128F09FC129F0D2
:101FC000A0C12AF00AEC2EF07EEC2FF028C0DEFF34
:101FD00029C0DDFF010EDBCF42F5DFCF43F52C6AD0
:101FE0002D6A2E6A3F0E2F6E99C127F09AC128F0F4
:101FF0009BC129F09CC12AF00AEC2EF07EEC2FF058
:1020000028C0DEFF29C0DDFF010EDBCF44F5DFCFA6
:1020100045F563C046F562C047F561C048F560C04C
:1020200049F563C04AF562C04BF561C04CF560C02C
:102030004DF5FDC14EF5FCC14FF52C6A2D6A2E6A97
:102040003F0E2F6E8DC127F08EC128F08FC129F071
:1020500090C12AF00AEC2EF07EEC2FF028C0DEFFB3
:1020600029C0DDFF010EDBCF50F5DFCF51F52C6A23
:102070002D6A2E6A3F0E2F6EB7C027F0B8C028F029
:10208000B9C029F0BAC02AF00AEC2EF07EEC2FF08D
:1020900028C0DEFF29C0DDFFDFCF52F52E0EDE6E39
:1020A000160EDD6E010EDBCF53F5DFCF54F5D20EE9
:1020B000DE6E040EDD6E010EDBCF55F5DFCF56F57B
:1020C000C20EDE6E010EDD6E010EDBCF57F5DFCFE7
:1020D00058F5BCC06EF0BDC06FF00501596BC5C0AE
:1020E0005AF5BEC06EF0BFC06FF005015B6BC6C095
:1020F0005CF5C0C06EF0C1C06FF06FC05DF56EC022
:102100005EF5C2C06EF0C3C06FF06FC05FF56EC009
:1021100060F555EC1DF079EF15F00101010EED6F42
:102120008B8055EC1DF079EF15F08B8E55EC1DF082
:1021300079EF15F00101ED6B8B9E55EC1DF079EFF9
:1021400015F00101010EF56FEBEC16F021EC17F024
:1021500055EC1DF079EF15F0EBEC16F033EC17F0C1
:1021600002C529F0E3EC2DF027C020F228C021F2AF
:1021700029C022F22AC023F22C6A2D6A800E2E6E0C
:10218000430E2F6E20C227F021C228F022C229F070
:1021900023C22AF0F3EC2EF027C000F028C001F093
:1021A00029C002F02AC003F003C529F0E3EC2DF0AA
:1021B00027C004F028C005F029C006F02AC007F0A7
:1021C00004C02CF005C02DF006C02EF007C02FF083
:1021D00000C027F001C028F002C029F003C02AF097
:1021E0000AEC2EF027C020F228C021F229C022F2EA
:1021F0002AC023F24AEC17F0400E0001B61100018C
:10220000B66F02C100F103C101F104C529F0E3EC8E
:102210002DF027C020F228C021F229C022F22AC0C6
:1022200023F22C6A2D6A800E2E6E430E2F6E20C272
:1022300027F021C228F022C229F023C22AF0F3ECB1
:102240002EF027C000F028C001F029C002F02AC0FB
:1022500003F005C529F0E3EC2DF027C004F028C0F9
:1022600005F029C006F02AC007F004C02CF005C014
:102270002DF006C02EF007C02FF000C027F001C0DF
:1022800028F002C029F003C02AF00AEC2EF027C083
:1022900020F228C021F229C022F22AC023F23EEC0B
:1022A00018F004C1E6FF04C100F005C101F0080EFA
:1022B0000F0B05E0D89001320032E806FBE1C00EBA
:1022C0000010E66EE4EC15F0E552E5520001B6AB05
:1022D00002D021EC17F055EC1DF079EF15F0EBEC86
:1022E00016F03CEC17F002C529F0E3EC2DF027C006
:1022F00020F228C021F229C022F22AC023F22C6A3F
:102300002D6A800E2E6E430E2F6E20C227F021C242
:1023100028F022C229F023C22AF0F3EC2EF027C0C5
:1023200000F028C001F029C002F02AC003F003C564
:1023300029F0E3EC2DF027C004F028C005F029C0F7
:1023400006F02AC007F004C02CF005C02DF006C02E
:102350002EF007C02FF000C027F001C028F002C007
:1023600029F003C02AF00AEC2EF027C020F228C082
:1023700021F229C022F22AC023F24AEC17F004C548
:1023800029F0E3EC2DF027C020F228C021F229C06B
:1023900022F22AC023F22C6A2D6A800E2E6E430E82
:1023A0002F6E20C227F021C228F022C229F023C2BA
:1023B0002AF0F3EC2EF027C000F028C001F029C06D
:1023C00002F02AC003F005C529F0E3EC2DF027C088
:1023D00004F028C005F029C006F02AC007F004C0A8
:1023E0002CF005C02DF006C02EF007C02FF000C065
:1023F00027F001C028F002C029F003C02AF00AEC3F
:102400002EF027C020F228C021F229C022F22AC0D3
:1024100023F23EEC18F00001B6AB02D021EC17F02D
:1024200055EC1DF066D3100EE66E79EC1DF0E5520A
:1024300060D3480EE66E79EC1DF0E5525AD3800E5B
:10244000E66E79EC1DF0E55254D374EC1DF065C0D6
:1024500041F564C042F50501436B70C044F56BC0A3
:1024600045F56AC046F567C047F566C048F508C13E
:10247000DEFF09C1DDFF010EDBCF49F5DFCF4AF5F5
:10248000BBC04BF555EC1DF034D374EC1DF003C507
:10249000BBF0BBC0E6FF080EE66E3AEC1DF0E5525D
:1024A000E55255EC1DF025D3A68E01C5F7FF02C5F8
:1024B000F6FFB4EC1FF00101F56B55EC1DF019D3DC
:1024C000F76AF66AA68EA684F29E010EDE6EDD6ABB
:1024D000DECF00F0DDCF01F0210E005C000E0158D0
:1024E00010E2DECFE9FFDDCFEAFF000EE926050EA0
:1024F000EA22EF50F56E0D00DF2A010E01E3DB2A20
:10250000E7D73EC5F7FF3FC5F6FF550EA76EAA0EEB
:10251000A76EA682F28EA69455EC1DF0EAD201C5F4
:1025200029F0E3EC2DF027C0E5F128C0E6F129C041
:10253000E7F12AC0E8F12C6A2D6A800E2E6E430E58
:102540002F6EE5C127F0E6C128F0E7C129F0E8C108
:102550002AF0F3EC2EF027C000F028C001F029C0CB
:1025600002F02AC003F002C529F0E3EC2DF027C0E9
:1025700004F028C005F029C006F02AC007F004C006
:102580002CF005C02DF006C02EF007C02FF000C0C3
:1025900027F001C028F002C029F003C02AF00AEC9D
:1025A0002EF027C0E5F128C0E6F129C0E7F12AC0E6
:1025B000E8F103C529F0E3EC2DF027C0E1F128C0D4
:1025C000E2F129C0E3F12AC0E4F12C6A2D6A800E01
:1025D0002E6E430E2F6EE1C127F0E2C128F0E3C159
:1025E00029F0E4C12AF0F3EC2EF027C000F028C057
:1025F00001F029C002F02AC003F004C529F0E3EC81
:102600002DF027C004F028C005F029C006F02AC02C
:1026100007F004C02CF005C02DF006C02EF007C056
:102620002FF000C027F001C028F002C029F003C03D
:102630002AF00AEC2EF027C0E1F128C0E2F129C00F
:10264000E3F12AC0E4F1EEEC18F03BC27EF53AC2A9
:102650007FF555EC1DF04DD2DE6ADD6ADECF00F06D
:10266000DDCF01F005013F51026E036A0250005CAC
:102670000350015823E2DECFE9FFDDCFEAFF010E70
:10268000E926000EEA22000EE926050EEA22EF50A6
:10269000E66E05013E51026E036ADE500224006EB2
:1026A000DD500320016E0050E66E3AEC1DF0E5525D
:1026B000E552DF2A010E01E3DB2AD0D705013C51A8
:1026C00001010A1501010A6F0B6B05013D51010162
:1026D0000A1101010A6F0BC10BF10AC1E6FF0F0ECF
:1026E000E66E3AEC1DF0E552E552A4EC1DF055EC17
:1026F0001DF0FFD10001B46B0001010EB56F3D0E5E
:102700000001B55D01E3C2D10001B551EA6A000FD5
:10271000E96E050EEA22EF50E66E0001B451EA6A56
:10272000B30FE96E010EEA22E552E750EF6E0001A9
:10273000B529EA6A000FE96E050EEA22EFCF00F034
:1027400000C029F0E3EC2DF027C020F228C021F2D0
:1027500029C022F22AC023F22C6A2D6A800E2E6E26
:10276000430E2F6E20C227F021C228F022C229F08A
:1027700023C22AF0F3EC2EF027C000F028C001F0AD
:1027800029C002F02AC003F0020E0001B525EA6A52
:10279000000FE96E050EEA22EFCF08F008C029F01D
:1027A000E3EC2DF027C004F028C005F029C006F0A6
:1027B0002AC007F004C02CF005C02DF006C02EF092
:1027C00007C02FF000C027F001C028F002C029F098
:1027D00003C02AF00AEC2EF027C020F228C021F214
:1027E00029C022F22AC023F20001B451EA6AB30FD1
:1027F000E96E010EEA22EF0435E11CC22CF01DC285
:102800002DF01EC22EF01FC22FF020C227F021C2D1
:1028100028F022C229F023C22AF009EC2EF027C0AA
:1028200000F028C001F029C002F02AC003F018C24D
:102830002CF019C22DF01AC22EF01BC22FF000C0CE
:1028400027F001C028F002C029F003C02AF0A0EC54
:102850002EF027C020F228C021F229C022F22AC07F
:1028600023F234D014C22CF015C22DF016C22EF073
:1028700017C22FF020C227F021C228F022C229F06F
:1028800023C22AF009EC2EF027C000F028C001F086
:1028900029C002F02AC003F010C22CF011C22DF0A2
:1028A00012C22EF013C22FF000C027F001C028F092
:1028B00002C029F003C02AF0A0EC2EF027C020F2BD
:1028C00028C021F229C022F22AC023F206C128F032
:1028D00007C129F0F4EC2DF027C000F028C001F06A
:1028E00029C002F02AC003F000C02CF001C02DF076
:1028F00002C02EF003C02FF020C227F021C228F022
:1029000022C229F023C22AF0B6EC2FF0010A0EE011
:1029100006C128F007C129F0F4EC2DF027C020F201
:1029200028C021F229C022F22AC023F206C128F0D1
:1029300007C129F0F4EC2DF027C004F028C005F001
:1029400029C006F02AC007F004C02CF005C02DF005
:1029500006C02EF007C02FF020C227F021C228F0B9
:1029600022C229F023C22AF0A0EC2EF027C000F0EA
:1029700028C001F029C002F02AC003F02C6AF00E32
:102980002D6E7F0E2E6E450E2F6E00C027F001C0FB
:1029900028F002C029F003C02AF0F3EC2EF027C083
:1029A00020F228C021F229C022F22AC023F22C6A88
:1029B0002D6A2E6A3F0E2F6E20C227F021C228F00A
:1029C00022C229F023C22AF00AEC2EF07EEC2FF06E
:1029D00028C000F029C001F00001B451E96EEA6A94
:1029E000D890E936EA36B90EE926010EEA2200C08F
:1029F000EEFF01C0EDFF050E0001B525EA6A000FEC
:102A0000E96E050EEA22070EEFCFDBFF060E00018E
:102A1000B525EA6A000FE96E050EEA22060EEFCF31
:102A2000DBFF070E0001B525EA6A000FE96E050E0F
:102A3000EA22050EEFCFDBFF080E0001B525EA6A9A
:102A4000000FE96E050EEA22040EEFCFDBFF000156
:102A5000B451040DF3CFE9FFF4CFEAFFC50EE92628
:102A6000010EEA22040EDBCFEEFF050EDBCFEEFFF8
:102A7000060EDBCFEEFF070EDBCFEEFF0001B42B1F
:102A80000A0E0001B5250001B56F39D63DC5B2F17A
:102A90000101050EB16F0101DD6BDE6BDF6BE06BD9
:102AA0009D80CD8055EC1DF024D0A68EA684A688EE
:102AB000F29E3EC5F7FF3FC5F6FF550EA76EAA0E64
:102AC000A76EA682F28EA69455EC1DF012D00501D9
:102AD000025101E080D90501035101E0B2D905019D
:102AE00004510101F36FF46BC9EC1FF055EC1DF0BC
:102AF00000D0400EE66E000EE66E050EE66EE66A4B
:102B0000010EE66EF6EC2CF0006E050EE15E005054
:102B1000F3CFE9F1F4CFEAF1080EE15C02E2E16AF9
:102B2000E552E16EE552E7CFD9FF1200D9CFE6FFBB
:102B3000E1CFD9FF030EE126DF6A010EDB6A020E48
:102B4000DB6A0001AE51DF5C1CE2C282C2B2FED77A
:102B5000C450056E046A010EDB500424026E020E9E
:102B6000DB500520036EC3500224006E000E0320CC
:102B7000016E010E00C0DBFF020E01C0DBFFDF2A89
:102B8000E0D7AE51006E016A010EDBCF28F0020ED5
:102B9000DBCF29F0AEC02DF001C02EF00DEC36F0E9
:102BA000F4EC2DF027C02EF228C02FF229C030F20D
:102BB0002AC031F2030EE15C02E2E16AE552E16E05
:102BC000E552E7CFD9FF1200D9CFE6FFE1CFD9FF19
:102BD0008B8CFE0EDB50800B800802E0000E01D0D3
:102BE000010EE8B08A8CE8A08A9C8A9E8A8EFE0E2E
:102BF000DB50400B400802E0000E01D0010EE8B0AF
:102C00008A8CE8A08A9C8A9E8A8EFE0EDB50200B5E
:102C1000200802E0000E01D0010EE8B08A8CE8A086
:102C20008A9C8A9E8A8EFE0EDB50100B100802E0F2
:102C3000000E01D0010EE8B08A8CE8A08A9C8A9E22
:102C40008A8EFE0EDB50080B080802E0000E01D051
:102C5000010EE8B08A8CE8A08A9C8A9E8A8EFE0EBD
:102C6000DB50040B040802E0000E01D0010EE8B0B6
:102C70008A8CE8A08A9C8A9E8A8EFE0EDB50020B0C
:102C8000020802E0000E01D0010EE8B08A8CE8A034
:102C90008A9C8A9E8A8EFE0EDB50010B010802E0A0
:102CA000000E01D0010EE8B08A8CE8A08A9C8A9EB2
:102CB0008A8EFD0EDB50800B800802E0000E01D0F2
:102CC000010EE8B08A8CE8A08A9C8A9E8A8EFD0E4E
:102CD000DB50400B400802E0000E01D0010EE8B0CE
:102CE0008A8CE8A08A9C8A9E8A8EFD0EDB50200B7F
:102CF000200802E0000E01D0010EE8B08A8CE8A0A6
:102D00008A9C8A9E8A8EFD0EDB50100B100802E012
:102D1000000E01D0010EE8B08A8CE8A08A9C8A9E41
:102D20008A8EFD0EDB50080B080802E0000E01D071
:102D3000010EE8B08A8CE8A08A9C8A9E8A8EFD0EDD
:102D4000DB50040B040802E0000E01D0010EE8B0D5
:102D50008A8CE8A08A9C8A9E8A8EFD0EDB50020B2C
:102D6000020802E0000E01D0010EE8B08A8CE8A053
:102D70008A9C8A9E8A8EFD0EDB50010B010802E0C0
:102D8000000E01D0010EE8B08A8CE8A08A9C8A9ED1
:102D90008A8E8B9CE552E7CFD9FF12000001A92B48
:102DA000AC51A95D03E1010EAD6FA96B0101B251F8
:102DB00001E0CD800001AF5105E0602B000E6123E2
:102DC00062236323AA2B4C0EAA5D04E1010EAB6FB4
:102DD000AA6BCD901200CD909D900101B26BE66A76
:102DE000800EE66EF1DEE552E552E66AC00EE66E52
:102DF000EBDEE552E55202012D6B0001AF6B0201E3
:102E0000366B376B2C6B0001AA6BB46B070EB45D8D
:102E100011E2B451080DF3CFE9FFF4CFEAFF710ED0
:102E2000E926000EEA22030EE926000EEA22EF6AE6
:102E3000B42BECD78A888A8A8998899A8B9EB06B42
:102E400012000001606B616B626B636B0101A16B2F
:102E5000A26BA36BA46B0101FC6BFD6B1200BBDFCB
:102E60008988898A12000101F55101E089888A98D0
:102E70000201010E2C6F12000101F55101E0898A57
:102E80008A9A02012C69E668CF0EE66E9DDEE55255
:102E9000E552120006C52DF201C5B6F006C128F0B4
:102EA00007C129F0F4EC2DF027C000F028C001F094
:102EB00029C002F02AC003F027C02CF028C02DF052
:102EC00029C02EF02AC02FF020C227F021C228F0FE
:102ED00022C229F023C22AF0B6EC2FF0010A0EE03C
:102EE00006C128F007C129F0F4EC2DF027C020F22C
:102EF00028C021F229C022F22AC023F202012D515A
:102F000059E12C0523E01CC22CF01DC22DF01EC27D
:102F10002EF01FC22FF020C227F021C228F022C2BB
:102F200029F023C22AF009EC2EF027C000F028C0B7
:102F300001F029C002F02AC003F018C22CF019C217
:102F40002DF01AC22EF01BC22FF022D014C22CF08A
:102F500015C22DF016C22EF017C22FF020C227F096
:102F600021C228F022C229F023C22AF009EC2EF057
:102F700027C000F028C001F029C002F02AC003F0E9
:102F800010C22CF011C22DF012C22EF013C22FF07D
:102F900000C027F001C028F002C029F003C02AF0C9
:102FA000A0EC2EF027C020F228C021F229C022F286
:102FB0002AC023F206C128F007C129F0F4EC2DF055
:102FC00027C004F028C005F029C006F02AC007F089
:102FD00027C02CF028C02DF029C02EF02AC02FF0D9
:102FE00020C227F021C228F022C229F023C22AF0F1
:102FF000A0EC2EF027C000F028C001F029C002F09C
:103000002AC003F02C6AF00E2D6E7F0E2E6E450E38
:103010002F6EF3EC2EF027C020F228C021F229C039
:1030200022F22AC023F22C6A2D6A2E6A3F0E2F6EDE
:103030000AEC2EF07EEC2FF028C002F129C003F13B
:1030400028C0E6FF28C000F029C001F0080E0F0BD1
:1030500005E0D89001320032E806FBE1800E001056
:10306000E66EB2DDE552E5520001010EAF6F400E93
:10307000B06F03C17EF502C17FF5120008C128F0D0
:1030800009C129F0F4EC2DF027C000F028C001F0B0
:1030900029C002F02AC003F027C02CF028C02DF070
:1030A00029C02EF02AC02FF020C227F021C228F01C
:1030B00022C229F023C22AF0B6EC2FF0010A0EE05A
:1030C00008C128F009C129F0F4EC2DF027C020F246
:1030D00028C021F229C022F22AC023F202012D5178
:1030E0002CE128C22CF029C22DF02AC22EF02BC2CE
:1030F0002FF020C227F021C228F022C229F023C2DB
:103100002AF009EC2EF027C000F028C001F029C0F9
:1031100002F02AC003F024C22CF025C22DF026C2F2
:103120002EF027C22FF0A0EC2EF027C020F228C0EE
:1031300021F229C022F22AC023F208C128F009C1D5
:1031400029F0F4EC2DF027C004F028C005F029C0C8
:1031500006F02AC007F027C02CF028C02DF029C0A7
:103160002EF02AC02FF020C227F021C228F022C260
:1031700029F023C22AF0A0EC2EF027C000F028C0CE
:1031800001F029C002F02AC003F02C6AF00E2D6E67
:103190007F0E2E6E450E2F6EF3EC2EF027C020F220
:1031A00028C021F229C022F22AC023F22C6A2D6AFB
:1031B0002E6A3F0E2F6E0AEC2EF07EEC2FF028C008
:1031C00004F129C005F10101FF0ED88028540F0E2B
:1031D000295403E204690F0E056F1200D9CFE6FFF0
:1031E000E1CFD9FF080EE126F6DD46DEE5C120F28B
:1031F000E6C121F2E7C122F2E8C123F24BDE67EC1F
:103200001DF079D99DC1DFFF010E9EC1DBFF020ECB
:103210009FC1DBFF030EA0C1DBFFE1C120F2E2C1D1
:1032200021F2E3C122F2E4C123F234DE67EC1DF0A7
:1032300062D9040E9DC1DBFF050E9EC1DBFF060EA9
:103240009FC1DBFF070EA0C1DBFFC5DD040EDBCF96
:1032500004F0050EDBCF05F0060EDBCF06F0070EFF
:10326000DBCF07F0D9CFE9FFDACFEAFFEECF08F0E6
:10327000EECF09F0EECF0AF0EFCF0BF008C02CF044
:1032800009C02DF00AC02EF00BC02FF004C027F0AB
:1032900005C028F006C029F007C02AF009EC2EF07E
:1032A00027C000F028C001F029C002F02AC003F0B6
:1032B000E1C12CF0E2C12DF0E3C12EF0E4C12FF00A
:1032C000E5C127F0E6C128F0E7C129F0E8C12AF0FE
:1032D00009EC2EF027C00CF028C00DF029C00EF02C
:1032E0002AC00FF027C02CF028C02DF029C02EF0E6
:1032F0002AC02FF000C027F001C028F002C029F03A
:1033000003C02AF0A0EC2EF027C020F228C021F242
:1033100029C022F22AC023F22C6A400E2D6E1C0E08
:103320002E6E460E2F6EF3EC2EF027C020F228C032
:1033300021F229C022F22AC023F2BBC029F0E3EC1B
:103340002DF0040E27C0DBFF050E28C0DBFF060EA4
:1033500029C0DBFF070E2AC0DBFF040EDBCF00F025
:10336000050EDBCF01F0060EDBCF02F0070EDBCF40
:1033700003F02C6A2D6A200E2E6E410E2F6E00C0B7
:1033800027F001C028F002C029F003C02AF0F3ECB6
:103390002EF0040E27C0DBFF050E28C0DBFF060E53
:1033A00029C0DBFF070E2AC0DBFF040EDBCF00F0D5
:1033B000050EDBCF01F0060EDBCF02F0070EDBCFF0
:1033C00003F020C22CF021C22DF022C22EF023C225
:1033D0002FF000C027F001C028F002C029F003C080
:1033E0002AF0ADEC2FF0010A04E102013A6B3B6BCD
:1033F00033D0040EDBCF04F0050EDBCF05F0060E54
:10340000DBCF06F0070EDBCF07F004C02CF005C0C1
:103410002DF006C02EF007C02FF020C227F021C2E9
:1034200028F022C229F023C22AF009EC2EF027C08E
:1034300000F028C001F029C002F02AC003F02C6A75
:103440002D6A2E6A3F0E2F6E0AEC2EF07EEC2FF0C6
:1034500028C03AF229C03BF2080EE15C02E2E16AC0
:10346000E552E16EE552E7CFD9FF120032C22CF0EF
:1034700033C22DF034C22EF035C22FF09DC127F09B
:103480009EC128F09FC129F0A0C12AF0B6EC2FF010
:10349000010A08E1020E0201365D02E1020E376FF9
:1034A000362B12000201366B12000001B36B080EBE
:1034B000B35D20E2B451080DF3CF00F0F4CF01F07A
:1034C000710E0026000E0122B3510F010024E96E97
:1034D000000E0120EA6EEF50E66E0001B551B52BEB
:1034E000EA6A400FE96E050EEA22E552E750EF6EF8
:1034F000B32BDDD71200D9CFE6FFE1CFD9FF020E03
:10350000E126210EC26E96EC15F00001B251C45CAA
:103510000FE0C4CFB2F0CD90E66AB2C0E6FFE4ECB3
:1035200015F0E552E5520101B25101E0CD80CFDA4C
:10353000010EC26E96EC15F0B2C029F0E3EC2DF04E
:1035400027C09DF128C09EF129C09FF12AC0A0F19B
:103550002C6A2D6A800E2E6E450E2F6EF3EC2EF027
:1035600027C000F028C001F029C002F02AC003F0F3
:103570002EC22CF02FC22DF030C22EF031C22FF00F
:103580000AEC2EF027C09DF128C09EF129C09FF1C2
:103590002AC0A0F191C12CF092C12DF093C12EF060
:1035A00094C12FF0F3EC2EF027C09DF128C09EF1BE
:1035B00029C09FF12AC0A0F102012D5152E1000162
:1035C000B251040DF3CFE9FFF4CFEAFF4C0EE92628
:1035D000010EEA22EECF04F0EECF05F0EECF06F0BA
:1035E000EFCF07F004C02CF005C02DF006C02EF080
:1035F00007C02FF09DC127F09EC128F09FC129F080
:10360000A0C12AF009EC2EF027C000F028C001F07C
:1036100029C002F02AC003F00001B251040DF3CF1B
:10362000E9FFF4CFEAFF0C0EE926010EEA22EECF05
:1036300008F0EECF09F0EECF0AF0EFCF0BF008C0A4
:103640002CF009C02DF00AC02EF00BC02FF0A0EC1A
:103650002EF027C09DF128C09EF129C09FF12AC0FD
:10366000A0F1020EE15C02E2E16AE552E16EE55290
:10367000E7CFD9FF1200D9CFE6FFE1CFD9FF040E83
:10368000E12696EC15F0046A400E056E1C0E066EDF
:10369000450E076E2EC22CF02FC22DF030C22EF038
:1036A00031C22FF004C027F005C028F006C029F071
:1036B0002A6EF3EC2EF027C000F028C001F029C0DC
:1036C00002F02AC003F00C6AF00E0D6E7F0E0E6E33
:1036D000450E0F6E2EC22CF02FC22DF030C22EF0F0
:1036E00031C22FF00CC027F00DC028F00EC029F019
:1036F0002A6E09EC2EF027C008F028C009F029C076
:103700000AF02AC00BF027C02CF028C02DF029C0E9
:103710002EF02AC02FF000C027F001C028F002C010
:1037200029F003C02AF0A0EC2EF027C02EF228C00A
:103730002FF229C030F22AC031F22C6A400E2D6ED1
:103740001C0E2E6E460E2F6EA0EC2EF027C000F041
:1037500028C001F029C002F02AC003F027C0E6FF0C
:1037600028C0E6FF29C0E6FF2AC0E6FF9AEC30F049
:10377000E552E552E552E55226C0DEFF27C0DEFFE6
:1037800028C0DEFF29C0DDFFDD52DD52006A016A7C
:10379000800E026E3F0E036E0D0E106ECF0E116E78
:1037A0005B0E126E3B0E136EF10E276EBB0E286E73
:1037B000860E296E390E2A6E000EDFCF2CF0010E18
:1037C000DBCF2DF0020EDBCF2EF0030EDBCF2FF080
:1037D000F3EC2EF027C014F028C015F029C016F025
:1037E0002AC017F027C02CF028C02DF029C02EF0D9
:1037F0002AC02FF010C027F011C028F012C029F005
:1038000013C02AF00AEC2EF027C00CF028C00DF0EF
:1038100029C00EF02AC00FF07E0E276ED50E286E3E
:103820002F0E296E360E2A6E000EDFCF2CF0010E01
:10383000DBCF2DF0020EDBCF2EF0030EDBCF2FF00F
:10384000F3EC2EF0000EDFCF2CF0010EDBCF2DF0CD
:10385000020EDBCF2EF0030EDBCF2FF0F3EC2EF0B9
:1038600027C018F028C019F029C01AF02AC01BF090
:1038700027C02CF028C02DF029C02EF02AC02FF030
:103880000CC027F00DC028F00EC029F00FC02AF0A0
:103890000AEC2EF027C008F028C009F029C00AF071
:1038A0002AC00BF06A0E276E130E286E890E296E41
:1038B000330E2A6E000EDFCF2CF0010EDBCF2DF081
:1038C000020EDBCF2EF0030EDBCF2FF0F3EC2EF049
:1038D000000EDFCF2CF0010EDBCF2DF0020EDBCF80
:1038E0002EF0030EDBCF2FF0F3EC2EF0000EDFCF27
:1038F0002CF0010EDBCF2DF0020EDBCF2EF0030EED
:10390000DBCF2FF0F3EC2EF027C01CF028C01DF009
:1039100029C01EF02AC01FF027C02CF028C02DF0AF
:1039200029C02EF02AC02FF008C027F009C028F0C7
:103930000AC029F00BC02AF00AEC2EF027C004F0D0
:1039400028C005F029C006F02AC007F027C02CF0D7
:1039500028C02DF029C02EF02AC02FF000C027F07B
:1039600001C028F002C029F003C02AF0A0EC2EF01C
:1039700027C02EF228C02FF229C030F22AC031F21F
:10398000330E2C6E930E2D6E880E2E6E430E2F6E00
:1039900009EC2EF027C000F028C001F029C002F089
:1039A0002AC003F02C6A2D6A200E2E6E410E2F6E57
:1039B000F3EC2EF027C02EF228C02FF229C030F2EF
:1039C0002AC031F2040EE15C02E2E16AE552E16EE6
:1039D000E552E7CFD9FF1200EEC12CF0EFC12DF078
:1039E000F0C12EF0F1C12FF08DC127F08EC128F06B
:1039F0008FC129F090C12AF0ADEC2FF0010A2AE125
:103A0000EEC12CF0EFC12DF0F0C12EF0F1C12FF07E
:103A10008DC127F08EC128F08FC129F090C12AF006
:103A200009EC2EF027C000F028C001F029C002F0F8
:103A30002AC003F02C6A2D6A2E6A400E2F6EF3EC1A
:103A40002EF027C0B7F028C0B8F029C0B9F02AC0BE
:103A5000BAF005D00001B76BB86BB96BBA6B8DC10A
:103A6000EEF18EC1EFF18FC1F0F190C1F1F10101E2
:103A7000F76B1200D9CFE6FFE1CFD9FFFE0EDB5086
:103A8000A96EFD0EDB50A86EA69EA684F29E550E72
:103A9000A76EAA0EA76EA682A1A8FED7A198F28E45
:103AA000A694E552E7CFD9FF1200400EE66E400E15
:103AB000E66E050EE66E010EE66EE66EF6EC2CF096
:103AC000050EE15EF3CFEBF1F4CFECF11200020151
:103AD000386B396B100E385D270E395904E2382BDC
:103AE000000E3923F7D7120001C5ACF002C5AEF0C5
:103AF0001200D9CFE6FFE1CFD9FFE652A69EFE0E17
:103B0000DB50A96EDF6ADFCF00F0380EE76E0018D9
:103B1000E8AE02D0E73402D0E750005C0FE2A680A6
:103B2000A92ADFCFE9FFEA6AE9BEEA68400EE92682
:103B3000050EEA22A8CFEFFFDF2AE5D7B6DFE55270
:103B4000E552E7CFD9FF1200D9CFE6FFE1CFD9FF89
:103B5000E65201010A51040B02E0200E01D0740E5E
:103B6000DF6E0001B36B100EB35D49E2040EB303C8
:103B7000F350DF24E66ED8D8E55226C000F027C007
:103B800001F028C002F029C003F00001B351040D78
:103B9000F3CFE9FFF4CFEAFF0C0EE926010EEA228B
:103BA00026C0EEFF01C0EEFF02C0EEFF03C0EEFF35
:103BB000040EB303F3CF04F0020EDF24F324E66E09
:103BC000E4D8E55226C000F027C001F028C002F07A
:103BD00029C003F00001B351040DF3CFE9FFF4CF86
:103BE000EAFF4C0EE926010EEA2226C0EEFF01C0D4
:103BF000EEFF02C0EEFF03C0EEFFB32BB4D7400EC2
:103C0000DF24E66E91D8E55226C024F227C025F2C3
:103C100028C026F229C027F2420EDF24E66EB5D86E
:103C2000E55226C028F227C029F228C02AF229C06E
:103C30002BF201010A51020B02E0180E01D06C0EAA
:103C4000DF6EDFCFE6FF70D8E55226C008F227C04E
:103C500009F228C00AF229C00BF2020EDF24E66E38
:103C600094D8E55226C00CF227C00DF228C00EF2FF
:103C700029C00FF2040EDF24E66E56D8E55226C0A6
:103C800018F227C019F228C01AF229C01BF2060E3A
:103C9000DF24E66E7AD8E55226C01CF227C01DF25A
:103CA00028C01EF229C01FF201010A51010B02E0D7
:103CB000100E01D0640EDF6EDFCFE6FF35D8E5527F
:103CC00026C000F227C001F228C002F229C003F288
:103CD000020EDF24E66E59D8E55226C004F227C052
:103CE00005F228C006F229C007F2040EDF24E66EB2
:103CF0001BD8E55226C010F227C011F228C012F2DC
:103D000029C013F2060EDF24E66E3FD8E55226C026
:103D100014F227C015F228C016F229C017F2E55296
:103D2000E552E7CFD9FF1200D9CFE6FFE1CFD9FFA7
:103D3000FE0EDBCFE6FF29D8E55226C004F027C0EF
:103D400005F028C006F029C007F02C6A2D6A7A0E0B
:103D50002E6E440E2F6E26C027F005C028F006C038
:103D600029F007C02AF0A0EC2EF029C002F02AC0EA
:103D700003F027C026F028C027F029C028F02AC069
:103D800029F0E552E7CFD9FF1200D9CFE6FFE1CF06
:103D9000D9FF040EE126FE0EDB50A96EA69EA6807A
:103DA000A8CF29F0E3EC2DF027C0DEFF28C0DEFF0E
:103DB00029C0DEFF2AC0DDFFDD52DD52A92AA68020
:103DC000D9CFE9FFDACFEAFFEECF04F0EECF05F06E
:103DD000EECF06F0EFCF07F02C6A2D6A800E2E6E24
:103DE000430E2F6E04C027F005C028F006C029F04E
:103DF00007C02AF0F3EC2EF027C000F028C001F035
:103E000029C002F02AC003F0A8CF29F0E3EC2DF07E
:103E100027C008F028C009F029C00AF02AC00BF01A
:103E200027C02CF028C02DF029C02EF02AC02FF07A
:103E300000C027F001C028F002C029F003C02AF01A
:103E40000AEC2EF027C0DEFF28C0DEFF29C0DEFF0F
:103E50002AC0DDFFDD52DD52D9CFE9FFDACFEAFF1C
:103E6000EECF00F0EECF01F0EECF02F0EFCF03F097
:103E70002C6A2D6A2E6A470E2F6E00C027F001C0F3
:103E800028F002C029F003C02AF0ADEC2FF0010A9F
:103E900035E1D9CFE9FFDACFEAFFEECF04F0EECF7C
:103EA00005F0EECF06F0EFCF07F02C6A2D6A2E6AF0
:103EB000470E2F6E04C027F005C028F006C029F079
:103EC00007C02AF009EC2EF027C000F028C001F04E
:103ED00029C002F02AC003F02C6A2D6A800E2E6ED3
:103EE000BF0E2F6EF3EC2EF027C0DEFF28C0DEFFE2
:103EF00029C0DEFF2AC0DDFFDD52DD52D9CFE9FF48
:103F0000DACFEAFFEECF04F0EECF05F0EECF06F009
:103F1000EFCF07F02C6A2D6A200E2E6E410E2F6E09
:103F200004C027F005C028F006C029F007C02AF019
:103F3000A0EC2EF027C000F028C001F029C002F04C
:103F40002AC003F027C026F028C027F029C028F097
:103F50002AC029F0040EE15C02E2E16AE552E16E5A
:103F6000E552E7CFD9FF12000001200EB56F400ED9
:103F70000001B55D0DE209000001B551EA6A400F8C
:103F8000E96E050EEA22F5CFEFFF0001B52BEFD762
:103F90001200D9CFE6FFE1CFD9FFE652A68EF3C1DA
:103FA00000F0F4C101F00006000E015A030E0F0BE1
:103FB00005E0D89001320032E806FBE10050DF6EE8
:103FC000780EDF24F76EF3C100F0F4C101F00006B3
:103FD000000E015A050ED89000360136E806FBE1C6
:103FE0000050F66EC1DF60C5C4F069C5CEF06AC589
:103FF000CFF06BC5D0F06CC5D1F06DC5D2F06EC5F9
:10400000D3F06FC5D4F070C5D5F071C5D6F00001FE
:10401000C451050A01E154D1010A01E151D1070A55
:1040200001E145D1010A01E1B0D0030A01E048D124
:10403000EBEC16F033EC17F063C529F0E3EC2DF050
:1040400027C020F228C021F229C022F22AC023F280
:104050002C6A2D6A800E2E6E430E2F6EF3EC2EF01E
:1040600027C000F028C001F029C002F02AC003F0E8
:1040700064C529F0E3EC2DF027C004F028C005F05A
:1040800029C006F02AC007F027C02CF028C02DF068
:1040900029C02EF02AC02FF000C027F001C028F060
:1040A00002C029F003C02AF00AEC2EF027C020F24B
:1040B00028C021F229C022F22AC023F24AEC17F0CC
:1040C000400E0001B611B66F02C100F103C101F14B
:1040D00061C529F0E3EC2DF027C020F228C021F2C1
:1040E00029C022F22AC023F22C6A2D6A800E2E6E7D
:1040F000430E2F6EF3EC2EF027C000F028C001F025
:1041000029C002F02AC003F062C529F0E3EC2DF0CB
:1041100027C004F028C005F029C006F02AC007F027
:1041200027C02CF028C02DF029C02EF02AC02FF077
:1041300000C027F001C028F002C029F003C02AF017
:104140000AEC2EF027C020F228C021F229C022F26A
:104150002AC023F23EEC18F004C1E6FF04C100F0CF
:1041600005C101F0080E0F0B05E0D89001320032B6
:10417000E806FBE1C00E0010E66EE4EC15F0E55237
:10418000E5520001B6AB9CD08FD0EBEC16F03CECC6
:1041900017F063C529F0E3EC2DF027C020F228C00A
:1041A00021F229C022F22AC023F22C6A2D6A800E45
:1041B0002E6E430E2F6EF3EC2EF027C000F028C0B9
:1041C00001F029C002F02AC003F064C529F0E3EC35
:1041D0002DF027C004F028C005F029C006F02AC041
:1041E00007F027C02CF028C02DF029C02EF02AC0DF
:1041F0002FF000C027F001C028F002C029F003C052
:104200002AF00AEC2EF027C020F228C021F229C0A3
:1042100022F22AC023F24AEC17F061C529F0E3EC40
:104220002DF027C020F228C021F229C022F22AC096
:1042300023F22C6A2D6A800E2E6E430E2F6EF3EC45
:104240002EF027C000F028C001F029C002F02AC0DB
:1042500003F062C529F0E3EC2DF027C004F028C07C
:1042600005F029C006F02AC007F027C02CF028C0AE
:104270002DF029C02EF02AC02FF000C027F001C079
:1042800028F002C029F003C02AF00AEC2EF027C063
:1042900020F228C021F229C022F22AC023F23EECEB
:1042A00018F00001B6AB0CD021EC17F009D0EBEC04
:1042B00016F021EC17F00001010EAF6F400EB06F49
:1042C0000001C86BC96BCB6BCC6BE552E552E7CFF5
:1042D000D9FF12000001C82BCE5125E0CF51C85D97
:1042E00015E1C86BD051CB5D01E28988D051006ED9
:1042F000016AFE0E001803E1015001E1899ACB2BFF
:10430000040ED025D880CB5501E2CB6BCE51C85DD1
:104310000AE18998D051006E016AFE0E001803E18F
:10432000015001E1898ACA2BD45113E0D551CA5DED
:104330000CE1CA6BD651CD5D01E28B8ECD2B040E04
:10434000D625D880CD5501E2CD6BD451CA5D01E1AF
:104350008B9EC92BD15113E0D251C95D0CE1C96BC1
:10436000D351CC5D01E2898ACC2B040ED325D880B1
:10437000CC5501E2CC6BD151C95D01E1899A1200A3
:10438000090EC26EC282C2B2FED7C4500BE0010158
:10439000F6510BE00001D7510101F36FF46BF66B9E
:1043A000C9EF1FF00101010EF66F120002012C513E
:1043B000010A0BE0FE0A55E19DC12CF09EC12DF0D3
:1043C0009FC12EF0A0C12FF028D0ADC128F0AEC102
:1043D00029F0F4EC2DF027C008F028C009F029C01E
:1043E0000AF02AC00BF09DC12CF09EC12DF09FC198
:1043F0002EF0A0C12FF009EC2EF027C004F028C049
:1044000005F029C006F02AC007F027C02CF028C00C
:104410002DF029C02EF02AC02FF099C127F09AC1A3
:1044200028F09BC129F09CC12AF0F3EC2EF027C0A4
:1044300000F028C001F029C002F02AC003F02C6A65
:10444000500E2D6EC30E2E6E470E2F6EA0EC2EF06A
:1044500027C0A5F128C0A6F129C0A7F12AC0A8F15C
:1044600012000101A56BA66BA76BA86B12000101DE
:10447000DD51DE11DF11E01101E0C5D1B251B15DB6
:1044800002E2B12B01D0B16BB151040DF3CFE9FFC2
:10449000F4CFEAFFC50EE926010EEA22EECFDDF1E8
:1044A000EECFDEF1EECFDFF1EFCFE0F1B151EA6A0E
:1044B000B30FE96E010EEA22EF50030A01E18FD13A
:1044C000010A01E1DED0030A51E0010A01E09BD1BB
:1044D0000001B6AD30D0E66A800EE66EE4EC15F071
:1044E000E552E5528A8A899A33EC17F004C1E6FF57
:1044F00004C100F005C101F0080E0F0B05E0D890D3
:1045000001320032E806FBE1C00E0010E66EE4EC7A
:1045100015F0E552E55200C1E6FF00C100F001C10F
:1045200001F0080E0F0B01E152D1D8900132003298
:10453000E806FBE14CD1E66A800EE66EE4EC15F08D
:10454000E552E5528A8889983CEC17F002C1E6FFF3
:1045500002C100F003C101F0080E0F0B01E137D1D9
:10456000D89001320032E806FBE131D189AA24D08B
:10457000B151E96EEA6AD890E936EA36B90EE92611
:10458000010EEA22EF50E66EB151E96EEA6AD89068
:10459000E936EA36B90EE926010EEA22EECF00F03E
:1045A000EFCF01F0080E0F0B01E111D1D8900132CD
:1045B0000032E806FBE10BD189A83CD0E66A800E08
:1045C000E66EE4EC15F0E552E5520201386B396B0A
:1045D0000A0E385D000E395904E2382B000E3923DB
:1045E000F7D78A8889983CEC17F00101B151E96E40
:1045F000EA6AD890E936EA36B90EE926010EEA22CF
:10460000EF50E66EB151E96EEA6AD890E936EA36C3
:10461000B90EE926010EEA22EECF00F0EFCF01F04D
:10462000080E0F0B01E1D3D0D89001320032E8061A
:10463000FBE1CDD03CEC17F00101B151E96EEA6A23
:10464000D890E936EA36B90EE926010EEA22EF5093
:10465000E66EB151E96EEA6AD890E936EA36B90EEB
:10466000E926010EEA22EECF00F0EFCF01F0080EAE
:104670000F0B01E1ACD0D89001320032E806FBE12B
:10468000A6D089A824D0B151E96EEA6AD890E9365B
:10469000EA36B90EE926010EEA22EF50E66EB15174
:1046A000E96EEA6AD890E936EA36B90EE926010ED3
:1046B000EA22EECF00F0EFCF01F0080E0F0B01E180
:1046C00086D0D89001320032E806FBE180D089AA7A
:1046D00044D0E66A800EE66EE4EC15F0E552E55251
:1046E0008A8A899A33EC17F004C1E6FF04C100F00E
:1046F00005C101F0080E0F0B05E0D8900132003221
:10470000E806FBE1C00E0010E66EE4EC15F0E552A1
:10471000E5520101B151E96EEA6AD890E936EA360C
:10472000B90EE926010EEA22EF50E66EB151E96EAC
:10473000EA6AD890E936EA36B90EE926010EEA228D
:10474000EECF00F0EFCF01F0080E0F0B40E0D89055
:1047500001320032E806FBE13AD033EC17F004C135
:10476000E6FF04C100F005C101F0080E0F0B05E0E3
:10477000D89001320032E806FBE1C00E0010E66E70
:10478000E4EC15F0E552E5520101B151E96EEA6A37
:10479000D890E936EA36B90EE926010EEA22EF5042
:1047A000E66EB151E96EEA6AD890E936EA36B90E9A
:1047B000E926010EEA22EECF00F0EFCF01F0080E5D
:1047C0000F0B05E0D89001320032E806FBE1800EC5
:1047D0000010E66EE4EC15F0E552E55214D08A883C
:1047E0008A8A8998899AE66A800EE66EE4EC15F06A
:1047F000E552E552E66AC00EE66EE4EC15F0E552CD
:10480000E55202012C6BD880FF0E0101DD55FF0E31
:10481000DE55000EDF55000EE05507E2FF0EDD5FAE
:10482000DE5B000EDF5BE05B120000680168026A7D
:10483000036ADD0EE96E010EEA6EEE50005CDD6F7C
:10484000EE500158DE6FEE500258DF6FEE50035805
:10485000E06FDDC126F0DEC127F0DFC128F0296E50
:104860002B6A010E2C6E2D6A2E6ACFEC35F0265085
:10487000CF6EDDC1CEFF0101DD6BDE6BDF6BE06B68
:1048800012001200120012001200C4EF34F01200E5
:104890001E0EE66E010EE66E51EC2CF0E552E5526E
:1048A000400EE66E000EE66E050EE66EE66A010E3E
:1048B000E66EF6EC2CF0006E050EE15E0050F3CFD4
:1048C000E9F1F4CFEAF1120002015D0520E10201F5
:1048D0005E051DE1A09AD6DF6D9202015E6B0201BA
:1048E000100E3C6F0E0E3D6F3C07000E3D5B3C51C1
:1048F0003D11FAE16D84080E3C6F070E3D6F3C07D9
:10490000000E3D5B3C513D11FAE16D94A08A12000E
:10491000D9CFE6FFE1CFD9FFFD0EDBCF28F0FE0EA9
:10492000DBCF29F0050E281801E1295036E0E868B0
:10493000281802E17F0E29182FE0030E281801E144
:10494000295028E0020E281801E1295021E0010E2B
:10495000281801E129501AE0740E281801E12950A5
:1049600013E0750E281801E129500CE0730E281889
:1049700001E1295005E0720E28180FE129500DD0F1
:1049800082DF0BD07EDF09D07DDF07D081DF05D04D
:104990007EDF03D07ADF01D077DF010EE552E7CF6B
:0449A000D9FF120029
:0C49A400D9CFE6FFE1CFD9FFE652A09A80
:1049B0006A6A686A706A010EE66EE66AE66A710EF5
:1049C000E66E0F0EE66EF3EC35F0006E050EE15E5E
:1049D0000050160E6F6E9F0E6B6E7B0E696EDF6A57
:1049E000DF50006E016A080E005C000E015810E2F4
:1049F000DF50040DF3CFE9FFF4CFEAFF000EE92604
:104A0000040EEA22EE6AEE6AEE6AEE6ADF2AE8D760
:104A10006D8C6E6A6D986D9C68A607D068960201D1
:104A2000516B566B576B586BF7D70201010E686FCD
:104A3000696F6A6B6B6B5E6BDF6A020EDF5C26E28E
:104A4000EA6ADF34FE0BEA36E96E490EE926020E09
:104A5000EA22EE6AED6AEA6ADF34FE0BEA36E96EB4
:104A6000450EE926020EEA22EE6AED6ADF50EA6A96
:104A7000620FE96E020EEA22EF6ADF50EA6A640F03
:104A8000E96E020EEA22EF6ADF2AD7D70201080E8A
:104A9000496F040E4A6F160E706E0401200E026FED
:104AA000040E036F080E016F840E006F02013F6B4E
:104AB0003E6BE552E552E7CFD9FF1200D9CFE6FFB2
:104AC000E1CFD9FFE65202013E0507E16DBA05D0FC
:104AD000686A69806988020E3E6F6850040B05E0C1
:104AE0006950040B02E06894C6D86DB257D0685084
:104AF000010B09E06950010B06E054DFA08A0201B6
:104B0000040E3E6F68906850100B05E06950100B62
:104B100002E09CD8689868AC19D069AC0FD0010E3F
:104B2000E66EE66A000EE66EE66A730EE66EE66A0A
:104B300088EC24F0006E060EE15E0050689C0201D5
:104B4000665101E06607665101E148DB6850200BC1
:104B500004E06950200B01E060D86850020B13E0BC
:104B60006950020B10E0010EE66EE66A000EE66E7A
:104B7000E66AE6687F0EE66E88EC24F0006E060EAC
:104B8000E15E00506A6A040E0201E76E3E19E8AE6B
:104B900002D0E73402D0E7503E5D02E2A19A38D05D
:104BA00069A635D0DF6A040EDF5C31E268A62FD03B
:104BB0006CCF5FF202015F51780BE842E842E842B5
:104BC000606F68965FB506D06051EA6A640FE96E5F
:104BD000020E05D06051EA6A620FE96E020EEA2207
:104BE000EF70605102E15ED810D0000EE66EE66A0A
:104BF0005F0EE66E020EE66E720EE66EE66A88ECF8
:104C000024F0006E060EE15E0050DF2ACCD7A19A98
:104C1000E552E552E7CFD9FF120070A015D041C28E
:104C2000E9FF42C2EAFFEF5080080DE149C2E9FF07
:104C30004AC2EAFFEF50840806E141C2E9FF42C2DE
:104C4000EAFF8C0EEF6E7090689A12006984689883
:104C50006D820201010E5E6F000EE66EE66AE66E80
:104C6000E66A750EE66EE66A88EC24F0006E060EC3
:104C7000E15E0050120002015E6B000EE66EE66A15
:104C8000E66EE66A740EE66EE66A88EC24F0006E64
:104C9000060EE15E00506D92699468A402D068949B
:104CA000FCD71200D9CFE6FFE1CFD9FFE6520201CF
:104CB0002D0E666FFD0E5F1553E17E0E5F15E84009
:104CC0007F0B040DF3CF41F2F4CF42F2000E4127E7
:104CD000040E422341C243F242C244F2437541C230
:104CE000E9FF42C2EAFFEF503C0BE842E8420D0800
:104CF00035E1DF6A080EDF5C23E241C2E9FF42C210
:104D0000EAFF020EE926000EEA22EE50EFCFEAFF9C
:104D1000E96EEF50E66EDF50EA6A200FE96E040E8E
:104D2000EA22E552E750EF6E41C2E9FF42C2EAFFD4
:104D3000020EE926000EEA22EE2AEF22DF2ADAD757
:104D400041C2E9FF42C2EAFF020EE926000EEA2252
:104D5000200EEE6E040EED6E0DD807D03AD805D0B9
:104D6000FD0E5F15040801E159D8E552E552E7CF81
:104D7000D9FF120002014D6B676B6A6B6B6B616B45
:104D80004E6B49C2E9FF4AC2EAFFEF9E497549C22C
:104D9000E9FF4AC2EAFFEF9E497543C2E9FF44C2F8
:104DA000EAFFEF9E516B526B536B566B576B586B10
:104DB0008CD8000EE66EE66AE66EE66A030EE66ED4
:104DC000E66A88EC24F0006E060EE15E005034EFD7
:104DD0002AF0020E02014E5D02E1F4EF2AF04E6B62
:104DE00061511AE143C2E9FF44C2EAFFEE52080EE4
:104DF000EF6E43C2E9FF44C2EAFF020EE926000E4D
:104E0000EA22200EEE6E040EED6E43C2E9FF44C2AC
:104E1000EAFF8C0EEF6E1200616B1200D9CFE6FF35
:104E2000E1CFD9FFE65249C2E9FF4AC2EAFFEF509B
:104E3000400B01E0010EDF6E02014975080E3E5D78
:104E400008E122C46EFF6E5002E0100E01D0040E85
:104E50003E6F4E0526E149C2E9FF4AC2EAFF020E53
:104E6000E926000EEA22280EEE6E040EED6E5DDBE2
:104E7000020E02014D5D06E149C2E9FF4AC2EAFFA6
:104E8000840E0DD0DF5006E149C2E9FF4AC2EAFFB5
:104E9000C80E05D049C2E9FF4AC2EAFF880EEF6E8C
:104EA0000FD056AF0CD059515A1107E005D05AC255
:104EB000FAFF02015951F96EFADF0201569F4E6B5B
:104EC000E552E552E7CFD9FF120004012051600BF3
:104ED000E842E842E842E842E842000901E0120004
:104EE00021510C0A50E00B0A3FE00C0A31E0010AA4
:104EF00022E00B0A1EE0020A1CE0030A18E0080A7E
:104F000010E0010A0CE00F0A08E0030A01E01200B9
:104F10000201518F080E3E6F12007DEF29F093EFD2
:104F20002BF002013F0E4F6F020E506F0CD0DAEFE4
:104F300029F0C4EF27F0245102014F6F506B400E4F
:104F40004F27020E50235181010E526F518F1200D4
:104F50000201518F04012451EA6A400FE96E020EEA
:104F6000EA2222C4EFFF1200000EE66EE66AE66E49
:104F7000E66A020EE66EE66A88EC24F0006E060E23
:104F8000E15E005012001200D9CFE6FFE1CFD9FF59
:104F9000030EE1260401220510E120511F0B000938
:104FA0000CE10201518F030E0401215D04E10201B5
:104FB000010E5D6F02D002015D6B0401225101E020
:104FC00003D120511F0B020801E0FED024510F0B2A
:104FD000000901E1F9D024510F0B010801E2F4D0DE
:104FE000200E02013E5D01E0EFD0518F040124BF8D
:104FF00016D024510F0BE96EEA6AD890E936EA36EA
:10500000450EE926020EEA22EECFDEFFEDCFDDFFF0
:1050100024510F0BEA6A640FE96E020E15D0245179
:105020000F0BE96EEA6AD890E936EA36490EE926AE
:10503000020EEA22EECFDEFFEDCFDDFF24510F0B93
:10504000EA6A620FE96E020EEA22020EEFCFDBFF80
:10505000D950020FE96EDACFEAFFEF50010B03E1FE
:10506000000EDF9401D0DF8424BF0BD024510F0B3E
:10507000E96EEA6AD890E936EA36450EE926020E6C
:105080000AD024510F0BE96EEA6AD890E936EA3665
:10509000490EE926020EEA22DECFEEFFDDCFEDFF5C
:1050A000030E215D20E1DECFE9FFDDCFEAFFEF5007
:1050B000800B11E024BF07D024510F0BEA6A640F64
:1050C000E96E020E06D024510F0BEA6A620FE96EF8
:1050D000020EEA22EF82840EDECFE9FFDDCFEAFF87
:1050E000E850EF1271D0DF74DECFE9FFDDCFEAFFC9
:1050F000EF50800B1BE0DECFE9FFDDCFEAFFEF9E34
:10510000DECFE9FFDDCFEAFFEF8C020EE66EE66A46
:10511000DECFE6FFDDCFE6FF050EE66EE66A88EC41
:1051200024F0006E060EE15E005005D0DECFE9FFF0
:10513000DDCFEAFFEF8CDF74D950020FE96EDACFD2
:10514000EAFFEF50020B0EE1DECFE9FFDDCFEAFF11
:10515000EF50800B32E0DECFE9FFDDCFEAFFEF500A
:10516000040B2BE1040124BF07D024510F0BEA6A82
:10517000640FE96E020E06D024510F0BEA6A620F2B
:10518000E96E020EEA22EF923B0E006EDECFE9FFDF
:10519000DDCFEAFFE850EF16020EE66EE66ADECFDC
:1051A000E6FFDDCFE6FF050EE66EE66A88EC24F04A
:1051B000006E060EE15E005007D03B0EDECFE9FF29
:1051C000DDCFEAFFE850EF16030EE15C02E2E16A90
:1051D000E552E16EE552E7CFD9FF120002016851B6
:1051E0004DE1010E686F695149E1010E696F020ED0
:1051F0004E5D0DE149C2E9FF4AC2EAFFEE52EF6A95
:1052000049C2E9FF4AC2EAFFC80EEF6E12004E051E
:1052100035E1616B41C2E9FF42C2EAFFEE52080E7E
:10522000EF6E41C2E9FF42C2EAFF020EE926000E1C
:10523000EA22200EEE6E040EED6E41C2E9FF42C27C
:10524000EAFF840EEF6E010E616F43C2E9FF44C2B4
:10525000EAFFEE52080EEF6E43C2E9FF44C2EAFFD6
:10526000020EE926000EEA22200EEE6E040EED6E0E
:1052700043C2E9FF44C2EAFF800EEF6E1200020152
:105280006A6B6B6B020E4E5D18E143C2E9FF44C2CC
:10529000EAFFEE52080EEF6E43C2E9FF44C2EAFF96
:1052A000020EE926000EEA22280EEE6E040EED6EC6
:1052B00043C2E9FF44C2EAFF1DD052510401265DFA
:1052C000020153510401275904E226C452F227C4B3
:1052D00053F22BD949C2E9FF4AC2EAFF020EE9267E
:1052E000000EEA22280EEE6E040EED6E49C2E9FFB2
:1052F0004AC2EAFFC80EEF6E1200800E0401205D64
:1053000058E10201C00E516F04012351030A2FE03E
:10531000010A09E0030A4BE10201500E4F6F6A0EC9
:10532000506F120E3ED02251F66EF76AD890F636C4
:10533000F736F70EF6266A0EF7220900F5CF4FF280
:105340000A00F5CF50F2020E0201F76A4F25F66E01
:105350005051F7220800F5CF52F2030EF76A4F259D
:10536000F66E5051F7220800F5CF53F21200030EEB
:10537000225D1AE22251F66EF76AD890F636F736B9
:10538000F90EF6266A0EF7220900F5CF4FF20A0051
:10539000F5CF50F24FC2F6FF50C2F7FF0800F550AC
:1053A0000201526F536B12000201516B1200020195
:1053B000516B1200D9CFE6FFE1CFD9FF020EE126F3
:1053C0000401286B296B20511F0B020A11E0030A0C
:1053D0000CE0010A35E10201518F0401288102012C
:1053E0005D052EE1040128832BD00201518F28D0C6
:1053F0000201518F040124BF0BD024510F0BE96E21
:10540000EA6AD890E936EA36450EE926020E0AD055
:1054100024510F0BE96EEA6AD890E936EA36490E54
:10542000E926020EEA22EECFDEFFEDCFDDFFDECF72
:10543000E9FFDDCFEAFFEF50040B02E0010E286F19
:10544000020151AF07D0280E4F6F040E506F5181EB
:10545000020E526F020EE15C02E2E16AE552E16E79
:10546000E552E7CFD9FF12006D98020151BF2BD052
:1054700056AF09D0020E4E6F6B5101E100DF020101
:10548000696B686B120043C2E9FF44C2EAFFEE5247
:10549000080EEF6E43C2E9FF44C2EAFF020EE9269E
:1054A000000EEA22200EEE6E040EED6E43C2E9FFFE
:1054B00044C2EAFF8C0EEF6E49C2E9FF4AC2EAFF1E
:1054C000840EEF6E1200040120AF0DD00201010E18
:1054D0004E6F6A5101E1D3DE0201696B686B67515F
:1054E00023E1EEEF28F00201020E4E6F43C2E9FF06
:1054F00044C2EAFFEE52080EEF6E43C2E9FF44C217
:10550000EAFF020EE926000EEA22200EEE6E040EDD
:10551000ED6E43C2E9FF44C2EAFF840EEF6E696B91
:10552000686B675101E15ADE1200D9CFE6FFE1CF87
:10553000D9FFE652080EDF6E0201525D000E53598C
:105540000AE252C2DFFF4D5102E1010E03D04D05C8
:1055500002E1020E4D6FDF50016AE850525D526F5A
:1055600001505359536F49C2E9FF4AC2EAFFEE5254
:10557000DFCFEFFF280E5B6F040E5C6F51B118D0C8
:10558000DF502DE04FC2F6FF50C2F7FF4F2B000E49
:1055900050230800F550E66E5BC2E9FF5CC2EAFFEB
:1055A0005B2B000E5C23E552E750EF6EDF06E8D779
:1055B000DF5015E04FC2E9FF50C2EAFF4F2B000E4B
:1055C0005023EF50E66E5BC2E9FF5CC2EAFF5B2B43
:1055D000000E5C23E552E750EF6EDF06E9D7E55297
:1055E000E552E7CFD9FF1200D9CFE6FFE1CFD9FFCF
:1055F000020EE12641C2E9FF42C2EAFFEE52EFCFBE
:10560000DFFFDFCF00F000500201575D000E585958
:1056100002E257C2DFFFDF50006E016AE850575DBB
:10562000576F01505859586F010EDB6ADF50F36E07
:10563000010EDBCFF4FFF350F45C16E2010EDB50F9
:10564000EA6A280FE96E040EEA22EF50E66E54C2B1
:10565000E9FF55C2EAFF542B000E5523E552E750EF
:10566000EF6E010EDB2AE2D7000ED8805755000EF0
:10567000585527E243C2E9FF44C2EAFFEE52080E42
:10568000EF6E43C2E9FF44C2EAFF020EE926000EB4
:10569000EA22280EEE6E040EED6E41C2E9FF42C210
:1056A000EAFFEF50400B06E143C2E9FF44C2EAFFC4
:1056B000C80E05D043C2E9FF44C2EAFF880EEF6E70
:1056C00028D043C2E9FF44C2EAFFEE52080EEF6E53
:1056D00043C2E9FF44C2EAFF020EE926000EEA22B5
:1056E000200EEE6E040EED6E43C2E9FF44C2EAFFE7
:1056F000840EEF6E59515A1107E005D05AC2FAFFD5
:1057000002015951F96EFADF0201569F675101E11A
:1057100065DD020EE15C02E2E16AE552E16EE5520E
:10572000E7CFD9FF1200D9CFE6FFE1CFD9FFE6528C
:105730000201518F010EE66EE66AE66A710EE66EB0
:105740000F0EE66EF3EC35F0006E050EE15E0050D4
:10575000DF6ADF50006E016A080E005C000E01581F
:1057600010E2DF50040DF3CFE9FFF4CFEAFF000EA3
:10577000E926040EEA22EE6AEE6AEE6AEE6ADF2A93
:10578000E8D76D8C010EE66EE66AE66A400EE66EBC
:10579000020EE66EF3EC35F0006E050EE15E005091
:1057A0006D9C0201080E496F040E4A6F000E416F96
:1057B000040E426F41C243F2446F22C43FF23F5194
:1057C00002E1100E12D0010EE66EE66A3F0EE66EA2
:1057D000020EE66E010EE66EE66A88EC24F0006EBC
:1057E000060EE15E00500201200E3E6FE552E552CA
:1057F000E7CFD9FF1200D9CFE6FFE1CFD9FF020EE4
:10580000E126000EDE6E040EDD6EFD0EDB50E82498
:10581000026EFE0EDB50040DF3500224040DF4CF93
:1058200001F0D9CFE9FFDACFEAFFF350EE260150BD
:10583000ED22DECFE9FFDDCFEAFFEF9EFD0EDB506C
:105840000AE1FE0EEA6ADB34FE0BEA36E96E450E2B
:10585000E926020E09D0FE0EEA6ADB34FE0BEA36B8
:10586000E96E490EE926020EEA22DECFEEFFDDCF19
:10587000EDFFDECFE9FFDDCFEAFFEF9CDECFE9FFF2
:10588000DDCFEAFF040EE926000EEA22EF8C020EBD
:10589000E15C02E2E16AE552E16EE552E7CFD9FF51
:1058A0001200D9CFE6FFE1CFD9FF020EE126FD0EAF
:1058B000DBA407D0E66AFE0EDBCFE6FF9CDFE552F5
:1058C000E552FD0EDBA208D0010EE66EFE0EDBCF28
:1058D000E6FF91DFE552E552FE0EDB50016A700FE4
:1058E000006E0F0E012200C0DEFF01C0DDFFDECF23
:1058F000E9FFDDCFEAFFFD0EDBCFEFFF020EE15C3B
:1059000002E2E16AE552E16EE552E7CFD9FF12000B
:10591000D9CFE6FFE1CFD9FF020EE126FE0EDB5024
:1059200020E143C2E9FF44C2EAFFEE52080EEF6EE7
:1059300043C2E9FF44C2EAFF020EE926000EEA2252
:10594000200EEE6E040EED6E43C2E9FF44C2EAFF84
:105950008C0EEF6E49C2E9FF4AC2EAFF840EEF6E79
:105960003BD0FD0EDB50E824026EFE0EDB50040D32
:10597000F3500224040DF3CF00F0F4CF01F0000E39
:105980000026040E012200C0DEFF01C0DDFF840EF0
:10599000DECFE9FFDDCFEAFFE850EF12FD0EDB506E
:1059A000E824026EFE0EDB50040DF3500224010FBA
:1059B000040DF3CF00F0F4CF01F0000E0026040E2A
:1059C000012200C0DEFF01C0DDFF840EDECFE9FF53
:1059D000DDCFEAFFE850EF12020EE15C02E2E16A7D
:1059E000E552E16EE552E7CFD9FF1200D9CFE6FFCD
:1059F000E1CFD9FF020EE126FD0EDB500AE0FE0EDC
:105A0000EA6ADB34FE0BEA36E96E490EE926020E3D
:105A100009D0FE0EEA6ADB34FE0BEA36E96E450E6B
:105A2000E926020EEA22EECFDEFFEDCFDDFFD9CF71
:105A3000E9FFDACFEAFFEE50ED1003E1F36AF46A12
:105A400044D0DECFE9FFDDCFEAFF020EE926000EEB
:105A5000EA22FB0EDBCFEEFFFC0EDBCFEDFFDECF4D
:105A6000E9FFDDCFEAFFEE52FA0EDBCFEFFF400E8B
:105A7000DECFE9FFDDCFEAFFE850EF16880EDECF7C
:105A8000E9FFDDCFEAFFE850EF12FD0EDB500AE040
:105A9000FE0EEA6ADB34FE0BEA36E96E490EE926B1
:105AA000020E09D0FE0EEA6ADB34FE0BEA36E96E1E
:105AB000450EE926020EEA22EF74DECF00F0DDCFBC
:105AC00001F000C0F3FF01C0F4FF020EE15C02E24E
:105AD000E16AE552E16EE552E7CFD9FF1200D9CF76
:105AE000E6FFE1CFD9FF6DA84ED0FE0EEA6ADB34A7
:105AF000FE0BEA36E96E490EE926020EEA22EE5066
:105B0000EFCFEAFFE96E400EEE16EE6AEE6AEE6A3D
:105B1000FE0EEA6ADB34FE0BEA36E96E490EE92630
:105B2000020EEA22EE50EFCFEAFFE96EEE7CFE0EA7
:105B3000EA6ADB34FE0BEA36E96E490EE926020E0C
:105B4000EA22EF74400E006EFE0EEA6ADB34FE0BB2
:105B5000EA36E96E490EE926020EEA22EE50EFCF50
:105B6000EAFFE96E0050EF16FE0EEA6ADB34FE0B28
:105B7000EA36E96E490EE926020EEA22EE50EFCF30
:105B8000EAFFE96EEF7CE552E7CFD9FF12006D6ABC
:105B9000696A02013E6B120002013E5113E16D6A17
:105BA000696A160E6F6E9F0E6B6E7B0E696ED08EDD
:105BB000A28AA08AF28E6DB602D06D86FCD7020151
:065BC000010E3E6F120011
:0A5BC600219E05D0219E29AE02D0D9
:105BD000296C218E29C023F0226A336A326A860E2C
:105BE000246E256A30EF30F0219E08D0219E29AE28
:105BF00005D0286C291EE86A2922218E29C023F0AD
:105C000028C022F0336A326A8E0E246E256A30EF85
:105C100030F02F7E216A6CEC30F084EC30F021B64D
:105C200014EF30F021A20AD021AA03D021BE14EF34
:105C300030F021A420EF30F01DEF30F021AA05D084
:105C400021AC20EF30F01DEF30F021A00AD021A8C8
:105C500008D021BE04D021A402D029EF30F02DEFCE
:105C600030F0326A256A2F502A5C316E10E327C06B
:105C700033F028C022F029C023F02AC030F02CC015
:105C800027F02DC028F02EC029F0213A09D02CC0D1
:105C900033F02DC022F02EC023F02FC030F0316C35
:105CA000219E21BC218E30C024F021B05CEF30F069
:105CB0001A0E31605CEF30F0246A2A6A21A408D001
:105CC000276C281E291E2A1EE86A282229222A2239
:105CD00021AC08D0336C221E231E241EE86A222227
:105CE00023222422266A315207E02A34293228321C
:105CF00027322632312EF9D7275033262850222238
:105D0000295023222A50242226C032F0219E24AE7C
:105D10000BD0326C331E221E231E241EE86A33224F
:105D2000222223222422218E24A006D0D8802332AE
:105D3000223233323232302A30C024F030EF30F0A9
:105D4000216A6CEC30F084EC30F021B614EF30F0C6
:105D500021A205D021BA14EF30F01BEF30F021BAA8
:105D600027EF30F021A005D021B814EF30F027EF55
:105D700030F021B81BEF30F0256A7F0E2A24246E04
:105D8000E86A25222F50245EE86A255A1A0E306EE2
:105D90002A6A326A336A226A236A2C50275E2D509F
:105DA000285A2E50295A000E2A5A09E72C50272625
:105DB0002D5028222E502922000E2A2201D0328A6C
:105DC000D8902736283629362A36D89032363336B8
:105DD00022362336302EE1D7295028102710D8A498
:105DE000328A30EF30F0216A6CEC30F084EC30F025
:105DF00021B614EF30F021A205D021B814EF30F015
:105E00001BEF30F021AA05D021B014EF30F01BEFCA
:105E100030F021B002D021A802D027EF30F0256A5F
:105E20002F502A24246EE86A25227E0E245EE86A1A
:105E3000255A326A336A226A236A2E502902F4CF25
:105E400023F0F3CF22F02D502902F3503326F450E3
:105E50002222000E23222E502802F3503326F45023
:105E60002222000E23222C502902F3503226F45015
:105E70003322000E222223222D502802F3503226F4
:105E8000F4503322000E222223222E502702F350F8
:105E90003226F4503322000E222223222C502802D4
:105EA000F4503226000E3322222223222D502702C4
:105EB000F4503226000E33222222232230EF30F01B
:105EC00028C032F028502D02F4CF27F0F3CF26F06F
:105ED00029502E02F4CF29F0F3CF28F02D02F350F1
:105EE0002726F4502822E86A292232502E02F35045
:105EF0002726F4502822E86A2922000C216A6CEC3B
:105F000030F021B688EF2FF021A20ED021B405D0B9
:105F10007F0E296EFF0E286E1FD0800E296E286A14
:105F20001BD0296A286A18D021B0FBD78F0E2A60AF
:105F3000EDD77E0E2A64F5D78E0E2A5C05E0D89048
:105F4000293228322A2AF8D721A406D0286C291E03
:105F5000E86A292229AEE5D71200BFEC2FF021B65E
:105F6000000C21B0000C21B4000C010CBFEC2FF090
:105F700021B6000C21B0000C21A4000C010C216AF8
:105F80006CEC30F084EC30F021B6120021AE08D079
:105F900021A004D021A802D021801200219012005B
:105FA0002F502A5C0BE12E50295C08E12D50285C13
:105FB00005E12C50275C02E121801200D8A002D01C
:105FC000218E10D02A502FC02AF02F6E29502EC0BB
:105FD00029F02E6E28502DC028F02D6E27502CC091
:105FE00027F02C6E2F502A5C10E0FF0F09E0219063
:105FF00021B403D021AE2184120021AE21941200DD
:106000002F2AD8902E322D322C322C50275E2D5034
:10601000285A2E50295A29BEEAD7D8902736283632
:1060200029362A2EF8D7C8D77F0E2A6EFF0E296E82
:10603000286E276E12007F0E21BEFF0E2A6E02D040
:106040007F0E2A6E800E296E286A276AF3D721AE4A
:1060500004D0800E2A6E296AF7D72A6A296AF4D7F3
:106060002350221033103210F8E025BEF0D723BEA3
:106070000CD024502510EBE0D8903236333622363F
:1060800023362406D8A02506F2D72550D4E12428AB
:10609000D2E032AE11D07F0E321402E133A00CD028
:1060A000332AE86A2222232207E3D88023322232CD
:1060B0003332242A2428BFE02450C9E033C027F01B
:1060C00022C028F02334296E24302A6E29322A9ED9
:1060D00021BE2A8E1AEF30F029362A3602E32184B7
:1060E000217E06E121802A6A296A286A276A12002D
:1060F0002A2803E0D88029321200D890293202E100
:1061000021821200218612002E362F3602E3218CC6
:10611000217E06E121882F6A2E6A2D6A2C6A1200E0
:106120002F2803E0D8802E321200D8902E32EAE1D8
:04613000218A1200AE
:0C613400D9CFE6FFDACFE6FFE1CFD9FFBC
:10614000E2CFDAFF260EE12402E3E168E652E16ED7
:10615000D950050FE1D9A9EC33F0006E060EE15CD1
:1061600002E2E16AE552E16E0050DF6E800EDF5C14
:1061700005E00B0EDB5012E0DF0410E0210E000101
:10618000E26FE36B010EDB68020EDB68030EDB6877
:106190007F0EF36E040EF3CFDBFF8FD1040EDF5CB6
:1061A0000EE13EDA010EEECFDBFF020EEECFDBFF9B
:1061B000030EEECFDBFF040EEECFDBFF7ED1DF045C
:1061C00010E1210E0001E26FE36B010EDB6A020EAB
:1061D000DB6A800EF36E030EF3CFDBFF040EDB6889
:1061E0006CD1D9500C0F98D917EC33F0006E060E15
:1061F000E15C02E2E16AE552E16E0050FA0E26C06F
:10620000DBFFFB0E27C0DBFFFC0E28C0DBFFFD0E13
:1062100029C0DBFFA6D9F30E2C6E040E2D6E350EB1
:106220002E6E3F0E87D9ADEC2FF0010A09E1B3D9EC
:1062300084D909EC2EF067D9EDD984D9ACD916D020
:106240000C0EDB060D0E01E2DB068BD92C6A2D6AE3
:106250002E6A3F0E6FD976D9160EDBCF04F0170EDB
:10626000DBCF05F0180EDBCF06F0190E66D9F3EC84
:106270002EF049D9CFD90AEC2EF01A0E27C0DBFF39
:106280001B0E28C0DBFF1C0E29C0DBFF1D0E2AC021
:10629000DBFF160EDBCF27F0170EDBCF28F0180E32
:1062A000DBCF29F0190EDBCF2AF01A0EDBCF2CF052
:1062B0001B0EDBCF2DF01C0EDBCF2EF01D0EDBCF27
:1062C0002FF0A0EC2EF01FD9120E27C0DBFF130E0B
:1062D00028C0DBFF140E29C0DBFF150E2AC0DBFF30
:1062E0004DD9120EDBCF2CF0130EDBCF2DF0140E98
:1062F000DBCF2EF0150E62D90E0E27C0DBFF0F0E7E
:1063000028C0DBFF100E29C0DBFF110E2AC0DBFF07
:106310003D0EF36E1E0EF3CFDBFF7E0EF36E1F0EEF
:10632000F3CFDBFF0D0EF36E200EF3CFDBFFBF0EBE
:10633000F36E210EF3CFDBFF0E0EDBCF00F00F0E5E
:10634000DBCF01F0100EDBCF02F0110EDBCF03F03C
:106350003A0E2C6E3F0E2D6ED40E2E6EC00EEAD865
:106360000AEC2EF0220E27C0DBFF230E28C0DBFF35
:10637000240E29C0DBFF250E2AC0DBFF0E0EDBCF6B
:1063800027F00F0EDBCF28F0100EDBCF29F0110E17
:10639000DBCF2AF01E0EDBCF2CF01F0EDBCF2DF053
:1063A000200EDBCF2EF0210E09D9220EDBCF2CF0F0
:1063B000230EDBCF2DF0240EDBCF2EF0250EDBCF0E
:1063C0002FF0A0EC2EF007D9120EDBCF00F0130E49
:1063D000DBCF01F0140EDBCF02F0150EDBCF03F0A4
:1063E000CDD8010EDBCF2CF0020EDBCF2DF0030E4B
:1063F000DBCF2EF0040EE2D827C004F028C005F051
:1064000029C006F02AC007F078D8046A800E056E0D
:10641000310E066E3F0E076EC9D827C008F028C09F
:1064200009F029C00AF02AC00BF0CCD8E1D8F3EC6F
:106430002EF069D8830E146E800E156E5E0E166EE9
:10644000B90E176EB3D827C018F028C019F029C0AC
:106450001AF02AC01BF0B6D814C027F015C028F0D7
:1064600016C029F017C02AF0F3EC2EF027C010F068
:1064700028C011F029C012F02AC013F0010EDBCFA2
:106480001CF0020EDBCF1DF0030EDBCF1EF0040E5E
:10649000DBCF1FF01CC02CF01DC02DF01EC02EF055
:1064A0001FC02FF00AEC2EF027C00CF028C00DF012
:1064B00029C00EF02AC00FF020D8010EDBCF00F06B
:1064C000020EDBCF01F0030EDBCF02F0040EDBCFB8
:1064D00003F000C026F001C027F002C028F003C07E
:1064E00029F0260EE15C02E2E16AE552E16EE55236
:1064F000E5CFDAFFE7CFD9FF120064D882D80AECE3
:106500002EF0EBEF32F027C000F028C001F029C0D8
:1065100002F02AC003F01200E66E000EDA20E66EEA
:106520007FD8EECFE6FFEECFE6FFEECFE6FFEFCF70
:10653000E6FF12002F6E01EF33F0DBCF07F06AD8D1
:10654000F8EF32F009EC2EF0160E27C0DBFF170E25
:1065500028C0DBFF180E29C0DBFF190E2AC0DBFFA5
:106560001200FA0EDBCF00F0FB0EDBCF01F0FC0EC9
:10657000DBCF02F0FD0EDBCF03F01200120EDBCFFB
:1065800027F0130EDBCF28F0140EDBCF29F0150E09
:10659000DBCF2AF01200FA0EDBCF04F0FB0EDBCFCC
:1065A00005F0FC0EDBCF06F0FD0E12000C0EDBCF6B
:1065B00028F00D0EDBCF29F0F6EF2DF0DBCF2FF01A
:1065C000F3EF2EF027C02CF028C02DF029C02EF0BC
:1065D0002AC02FF01200010E27C0DBFF020E28C0D8
:1065E000DBFF030E29C0DBFF040E2AC0DBFF120015
:1065F00004C027F005C028F006C029F007C02AF023
:10660000120000C027F001C028F002C029F003C02A
:106610002AF012002C6A2D6A2E6A3F0E2F6E12008D
:0E662000D950FA0FE96EFF0EDA20EA6E120072
:02662E00D9CFC2
:10663000E6FFDACFE6FFE1CFD9FFE2CFDAFF0C0EBB
:10664000E12402E3E168E652E16ED950FA0FE96E07
:10665000FF0EDA20EA6E010EEECFDBFF020EEECF68
:10666000DBFF030EEECFDBFF040EEECFDBFF63D8C4
:10667000D950010FE96E000EDA20EA6EEECFE6FF88
:10668000EECFE6FFEECFE6FFEFCFE6FFA9EC33F06B
:10669000006E060EE15C02E2E16AE552E16E005036
:1066A000DF6E850EDF1404E04DD8EE6AED6A23D06C
:1066B000090EDBCF00F00A0EDBCF01F0820E0026C0
:1066C000FF0E01223FD800C0EEFF01C0EDFF7E0E9D
:1066D000F36E090EF3CFDBFF0A0EDB6AD950010F10
:1066E000E66E000EDA20E66E26D837EC34F0E5527E
:1066F000E552E552E552010EDBCF00F0020EDBCF92
:1067000001F0030EDBCF02F0040EDBCF03F000C07C
:1067100026F001C027F002C028F003C029F00C0EBB
:10672000E15C02E2E16AE552E16EE552E5CFDAFFB3
:10673000E7CFD9FF1200D950050FE66E000EDA2020
:10674000E66E1200F80EDBCFE9FFF90EDBCFEAFFB1
:02675000120035
:0E675200D9CFE6FFDACFE6FFE1CFD9FFE2CFE5
:10676000DAFFE652006801687F0E026E036AD950B4
:10677000FA0FE96EFF0EDA20EA6EEE500016EE50C8
:106780000116EE500216EE5003166AD800C0EEFF56
:1067900001C0EEFF02C0EEFF03C0EEFFFD0EDB50B6
:1067A000800B02E0010E01D0000EE66E59D8060EF5
:1067B000E926000EEA22E552E750EF6EFC0EDBCF31
:1067C00000F0FD0EDBCF01F0D89000360136FC0E54
:1067D00000C0DBFFFD0E01C0DBFFDB50E66E40D8E2
:1067E000040EE926000EEA22E552E750EE6EED6A4D
:1067F000FD0EDB50006E016AFF0E001818E101501B
:1068000016E12ED8EECF00F0EECF01F0EECF02F081
:10681000EFCF03F0005001100210031006E0210E2C
:106820000001E26FE36B800E0BD0040E09D0FD0E69
:10683000DB5008E115D8EE6AEE6AEE6AEE6A010EE8
:10684000DF6E06D0020EDF6E0BD8EE52EE52EE8EE9
:10685000DF50E552E552E5CFDAFFE7CFD9FF12006E
:0E686000F80EDBCFE9FFF90EDBCFEAFF1200E6
:02686E00D9CF80
:10687000E6FFDACFE6FFE1CFD9FFE2CFDAFF5BD860
:10688000013411E20050FE08000E01540CE276D8EB
:1068900005E06CD8800EEE6EEE6847D067D8800EAB
:1068A000EE6E7F0E0ED047D8D890015004E6010E50
:1068B000005C000E01580BE261D805E057D8EE6A83
:1068C000800EEE6E32D052D8EE6AEE6A2ED047D8E5
:1068D000EECF00F0EECF01F0EECF02F0EFCF03F0FD
:1068E00032D800C0EEFF01C0EEFF02C0EEFF03C0D1
:1068F000EEFF21D80050010B05E025D8020E3AD852
:10690000EF8E04D020D8020E35D8EF9E14D8D89040
:106910000132003218D8030E2DD800C0EFFF1AD86C
:1069200004E011D8030E26D8EF8EE552E5CFDAFF4A
:10693000E7CFD9FF120013D8040E1CD8EECF00F019
:10694000EFCF01F01200FA0EDBCFE9FFFB0EDBCF39
:10695000EAFF120004D8060E0DD8EF501200FC0E0C
:10696000DBCFE9FFFD0EDBCFEAFF1200ECDFEE6AC2
:10697000EE6A1200E926000EEA221200220E000141
:08698000E26FE36BAAEF34F0B3
:08698800040120511F0B01085E
:1069900001E01200245101E01200060E215D1EE10B
:1069A0002351230A1BE0010A0CE0030A17E102014C
:1069B0003F0514E10201740E4F6F6A0E506F090E0D
:1069C00009D002013F050AE10201DB0E4F6F6A0E9A
:1069D000506F1C0E526F536BC00E516F040120514B
:1069E000600BE842E842E842E842E842010801E080
:1069F000120021510B0A26E0080A19E0090A11E0E9
:106A0000080A05E00B0A23E0080A21E0120002014F
:106A1000FE0E4F6F010E506F010E526F536BC10E81
:106A20000FD00201800E516F23C4FEF1120002014B
:106A3000FF0E4F6F010E506F010E526F536B810EA0
:106A4000516F12000201800E516F22C4FFF112003B
:106A50001201000200000008D80460FD03000102DA
:106A6000000109022900010100C0320904000002EE
:106A700003000000092111010001221C000705810B
:106A80000340000107050103400001040309041E3F
:106A900003420061007400740065007200790020F8
:106AA000004D00650074007200690063002E03420F
:106AB00000410035003000300020004200610074C9
:106AC000007400650072007900200041006E0061D2
:106AD000006C0079007A00650072000600FF090171
:106AE000A101190129401501254075089540810033
:0F6AF000190129409100C0626A8B6A8F6AAD6AF2
:106B00002A0EF66E100EF76E000EF86E00010900E8
:106B1000F550DD6F0900F550DE6F03E1DD6701D050
:106B20003DD00900F550D86F0900F550D96F090024
:106B3000F550DA6F09000900F550E96E0900F550CB
:106B4000EA6E090009000900F550DB6F0900F550F5
:106B5000DC6F09000900F6CFDFF0F7CFE0F0F8CFE7
:106B6000E1F0D8C0F6FFD9C0F7FFDAC0F8FF0001A6
:106B7000DB5302E1DC5307E00900F550EE6EDB0762
:106B8000F8E2DC07F9D7DFC0F6FFE0C0F7FFE1C0AD
:0E6B9000F8FF0001DD07000EDE5BBFD712002C
:026B9E00256A66
:106BA000246A236A226A200EE76ED890263627369A
:106BB0002836293622362336243625362B50225CB9
:106BC0002C5023582D5024582E50255809E32B5073
:106BD000225E2C50235A2D50245A2E50255A262AF4
:066BE000E72EE4D71200CD
:0A6BE600FE0EE3CFE9FFFF0EE3CF40
:106BF000EAFFE9CFF3FFEACFF4FFFB0EE35003E136
:106C0000FC0EE35009E0FB0EE30602E2FC0EE30695
:0A6C1000FD0EE350EE6EF1D7120006
:066C1A00256A246A100E39
:106C2000E76ED89028362936243625362D50245C38
:106C30002E50255805E32D50245E2E50255A282A23
:066C4000E72EF0D7120060
:0A6C460013EE00F023EE00F0F86AF0
:106C5000219C80EC35F038EC36F0C4EC08F0FBD722
:026C6000120020
:0E6C620000EE00F00F0EEE6AEA62FDD712009F
:026C7000120010
:0E6C7200000000000000007A44000100000055
:076C8000000000000000000D
:00000001FF
